:020000040000FA
:100000000002040000000000EA770000EA77000028
:10001000EA770000EA770000EA770000EA7700005C
:10002000EA770000EA770000EA770000EA7700004C
:10003000EA770000EA770000EA770000EA7700003C
:10004000EA770000EA770000EA770000EA7700002C
:10005000EA770000265B0000485B0000EA770000BA
:10006000EA770000EA770000EA770000EA7700000C
:10007000EA770000EA770000EA770000EA770000FC
:10008000EA770000EA770000EA770000EA770000EC
:10009000EA770000EA770000EA770000EA770000DC
:1000A000EA770000EA770000EA770000EA770000CC
:1000B000EA770000EA770000EA770000EA770000BC
:1000C000EA770000EA770000EA770000EA770000AC
:1000D000EA770000EA770000EA770000EA7700009C
:1000E000EA770000EA770000EA770000EA7700008C
:1000F000EA770000EA770000EA770000EA7700007C
:10010000EA770000EA770000EA770000EA7700006B
:10011000EA770000EA770000EA770000EA7700005B
:10012000EA770000EA770000EA770000EA7700004B
:10013000EA770000EA770000EA770000EA7700003B
:10014000EA770000EA770000EA770000EA7700002B
:10015000EA770000EA770000EA770000EA7700001B
:10016000EA770000EA770000EA770000EA7700000B
:10017000EA770000EA770000EA770000EA770000FB
:10018000EA770000EA770000EA770000EA770000EB
:10019000EA770000EA770000EA770000EA770000DB
:1001A000EA770000EA770000EA770000EA770000CB
:1001B000EA770000EA770000EA770000EA770000BB
:1001C000EA770000EA770000EA770000EA770000AB
:1001D000EA770000EA770000EA770000EA7700009B
:1001E000EA770000EA770000EA770000EA7700008B
:1001F000EA770000EA770000EA770000EA7700007B
:10020000FFFFFF00FFFFFF00EA770000EA77000032
:10021000EA770000EA770000EA770000EA7700005A
:10022000EA770000EA770000EA770000EA7700004A
:10023000EA770000EA770000EA770000EA7700003A
:10024000EA770000EA770000EA770000EA7700002A
:10025000EA770000265B0000485B0000EA770000B8
:10026000EA770000EA770000EA770000EA7700000A
:10027000EA770000EA770000EA770000EA770000FA
:10028000EA770000EA770000EA770000EA770000EA
:10029000EA770000EA770000EA770000EA770000DA
:1002A000EA770000EA770000EA770000EA770000CA
:1002B000EA770000EA770000EA770000EA770000BA
:1002C000EA770000EA770000EA770000EA770000AA
:1002D000EA770000EA770000EA770000EA7700009A
:1002E000EA770000EA770000EA770000EA7700008A
:1002F000EA770000EA770000EA770000EA7700007A
:10030000EA770000EA770000EA770000EA77000069
:10031000EA770000EA770000EA770000EA77000059
:10032000EA770000EA770000EA770000EA77000049
:10033000EA770000EA770000EA770000EA77000039
:10034000EA770000EA770000EA770000EA77000029
:10035000EA770000EA770000EA770000EA77000019
:10036000EA770000EA770000EA770000EA77000009
:10037000EA770000EA770000EA770000EA770000F9
:10038000EA770000EA770000EA770000EA770000E9
:10039000EA770000EA770000EA770000EA770000D9
:1003A000EA770000EA770000EA770000EA770000C9
:1003B000EA770000EA770000EA770000EA770000B9
:1003C000EA770000EA770000EA770000EA770000A9
:1003D000EA770000EA770000EA770000EA77000099
:1003E000EA770000EA770000EA770000EA77000089
:1003F000EA770000EA770000EA770000EA77000079
:10040000CFD621000E7F22000E01880000000000E0
:100410000C000700E03F260001002000110007004B
:10042000000020000000E000020032000000020096
:1004300000000000B8740200000000000040DA0074
:100440000000FE004440A900E01C20000000E00085
:100450000300320000002000A00188004440A800F2
:100460000000060091018800800078000000EB0089
:1004700015003700E280400032A0B4009101BA00BC
:10048000E280400032A0B4009102BA00E280400055
:1004900032A0B4000002EB00472BDE00F507B200EB
:1004A000602CE10004003A000059EB008301E900F0
:1004B000FDFF3E00040037006128E100010032002A
:1004C0000082EB00040007001101BA000200E00006
:1004D000E8FF3A00000006003159BA008301E90044
:1004E0000C0032002159BA008301E90008003200F3
:1004F0000400E00003003A00E280400032A0B400B3
:10050000F5FF370011D9BA008301E900FAFF3A007C
:100510008100E800E180400032A0B4000000060045
:1005200000000000000000000000000000000000CB
:1005300000000000000000000000000000000000BB
:1005400000000000000000000000000000000000AB
:10055000000000000000000000000000000000009B
:1007D000889FBE008A9FBE00010578000100E000EE
:1007E0000400350008003C000000E000200032005A
:1007F0000500370060001000E080180002003B0098
:1008000001F02C001A0037000004BE006011B8008F
:100810006B0920000982CF00020039000882CF0056
:100820000441B000694252000E00320008003B0053
:1008300082817100610164008904D1000884D300C1
:100840008B05E8000442E800F9FF3A000500370094
:100850000804440089844C008B05E9000442E90047
:10086000FBFF3A000B0107000AF0A70001F0A0000F
:100870004F05BE004F04BE0000000600F4FF2F002D
:100880002A0137001400200028013700889FBE008D
:100890008A9FBE008C1F78003F010700460133008D
:1008A00003866C006450E1002E0032006420E100F9
:1008B000330032006150E1002F0032006120E1007E
:1008C0003100320085855500EB07B000090020009B
:1008D00008042000050037000804440089844C0007
:1008E0000A0031000603430087834B0000015300D8
:1008F00081815B00F8FF33000203BE000800A00006
:100900000804440089844C00F6FF3900C639DD0034
:100910008301730001003200130020008904D1001C
:100920000884D3000998A300050032000800A7003E
:100930000300A0008904D1000884D3008B05E800DF
:100940008904D1000884D3000001EB000281D200A9
:10095000D000070001F0A1000CF0A70001F0A000FA
:100960001E0137006420E100200132000801BE00B2
:100970000200BE00F7FF37006120E1001B013200DA
:100980006000B800F3FF37000000200001F82700E6
:10099000F0FF370003F0A200889FBE008A9FBE00D0
:1009A0008C1F7800FC000700030133006450E10055
:1009B0004F0032006420E1005200320003826C00DC
:1009C00007003B000905D0000306D000820F540049
:1009D0000C065D0002003900020032008901780037
:1009E000030678008582550004003D000003FD00E9
:1009F0008103FD008502EA008B854200840F7200AE
:100A000002003B0060001000E08018006011B80098
:100A10000005EB007A28E1000A00390006007800A2
:100A2000C75DDD00F707B200878075002D00370035
:100A3000828171000A017800610560008180D10027
:100A40000080D3008502E900F9FF3B000604400066
:100A50008784480002003B0060041400E0841C000E
:100A60000988A300070032008A8171008281710029
:100A7000610164008904D1000884D3008B05E8007B
:100A8000170037000978A30013003A000B00E000BC
:100A9000130034008B05E9000804440089844C00ED
:100AA0000A4474000978A3000D003A000B00E0002E
:100AB000070034008B05E9000804440089844C00D9
:100AC00001003A000B0020000978A300F7FF320074
:100AD0000001EB0002003700828171000A017800FA
:100AE0006C0007000CF0A70001F0A000BB0037006D
:100AF0006420E10002003A00838F6C00BB003300E9
:100B00000801BE000200BE00B4003700889FBE008E
:100B10008A9FBE008C1F78009F000700A60033004C
:100B200003866C006450E100240032006420E10080
:100B3000270032006150E100220032006120E10014
:100B4000210032008B854200EB07B1000134B80070
:100B5000003AB8000804420089844A00013AB8000B
:100B60000030B8008880400009014A0004003300CA
:100B70000000400081804800020149008B05E90027
:100B8000C909DD008301700001003200130020005C
:100B9000C814DE004814DD004709DE001200B20070
:100BA000C808DE00088470003A00070001F0A100C8
:100BB0000CF0A70001F0A000880037006120E100E0
:100BC0008A0032000801BE000200BE00F7FF3700B5
:100BD0006150E100FCFF3A00840037000001BE00D4
:100BE000850007000470A70003F0A10003F8A3002C
:100BF00013003A006509B100100032000900350009
:100C00006928E1000200350001002800000005000D
:100C100000004000818048008502E900FCFF3A00A6
:100C200000000600F88F4200050035008100D10069
:100C30000080D3008502E800FCFF3A0000000600B7
:100C40008000EB00000005006022B80006022000D2
:100C50000000D0008180D2000482D2008582D200C0
:100C60000000A0000202520083825A0003003100FB
:100C70000202420083824A000000A1000603E9004C
:100C8000F3FF3A0000000600EFFF07000400BE007B
:100C90000000060081002000618055000B003D002F
:100CA0000B00200061FE2F000100E1001D00340058
:100CB00082817100610164008904D1000884D3003D
:100CC0000000E800FAFF3A007100200061006400B3
:100CD000030070000200600009003200610444005B
:100CE000E0844C000988A500050032008B05E8006F
:100CF0006808E10002003A008904D1000884D300AA
:100D0000F20F20000258E10005003D00C75DDD0044
:100D1000F907B2008980750008007800000006001D
:100D20000BF827008B00780000000500889FBE00AC
:100D30008A9FBE00841F7800170007004F007800CC
:100D400011003300F0FF2F00838F6C0006003B0082
:100D5000040565000A00A7000800370009F0A60096
:100D60001000200008003700820F5400838F5C00C1
:100D7000030039001000200001003E0000002000A8
:100D800009F0A7000000EA004F05BE004F04BE00B6
:100D90000000E000000006000004BE00160007008E
:100DA0000003BE000405BE000200BE0012000700E2
:100DB000844F7500000006000200BE006450E10090
:100DC000050036006420E100020036000968A30037
:100DD00001003A000800BE000160A0004F06780044
:100DE0004F05BE004F04BE0000000600F0FF2F00BC
:100DF000F1FF2700F9FF3700C70ADE00F107B20054
:100E0000F50FB20008003200E1CF420002003200CC
:100E10000170A00024000500810F70000100320065
:100E20000408050044000500810F700002003A002C
:100E3000140005008502E9000000400081C0480060
:100E4000FCFF3B000170A000240005003E000000F4
:100E500008200000080000001B5B000044000000A8
:100E60001B5B000000440000001B00005B4300000F
:100E7000001B00005B3200004B0D0000004300002F
:100E8000000000001B5B000032440000005700001F
:100E9000617200006E6900006E6700003A20000079
:100EA0006E6F0000207600006F6C0000746100001F
:100EB00067650000206F00006E2000005670000083
:100EC000756C00006C7500007020000070690000F7
:100ED0006E000000203D000020000000565200007F
:100EE00045470000207400006F6F0000206C000078
:100EF0006F7700002C200000697300002074000050
:100F00006865000072650000206100002073000029
:100F1000686F0000727400003F0000002E20000087
:100F20003C0000002E200000000D00000A280000F8
:100F300000780000002900003E000000427500001B
:100F400073200000506900007261000074650000A9
:100F50002076000033000000206300006C6F00006A
:100F60006E650000207700002F64000069660000B5
:100F700066650000726500006E740000205000007D
:100F80004943000000460000697200006D770000D0
:100F90006172000065200000763600002E320000ED
:100FA0002D620000657400006131000020720000B5
:100FB00031390000383100002000000020280000F6
:100FC00032340000464A0000363400004741000039
:100FD000303000000034000020000000322000000B
:100FE00000410000330000004234000000420000D5
:100FF0003500000042380000005500004E4B000054
:101000000029000000490000090000004F0900000D
:1010100000480000090000004C09000000450000E5
:101020006E7400006572000020720000617700009D
:1010300020760000616C00007565000020660000ED
:101040006F720000204200005247000000000000C4
:101050000000000000000000000000002C01000063
:10106000000000005802000000000000B004000072
:10107000000000006009000000000000C012000035
:101080000000000080250000000000004038000043
:1010900000000000004B0000000000008070000015
:1010A000000000000096000000000000C0DA000010
:1010B0000000000000E100000000000000C200008D
:1010C0000100000000F400000100000000E8000042
:1010D00003000000415200005431000000000000F5
:1010E0003062000000300000303000002C000000B2
:1010F0003030000000300000313200003334000096
:101100003536000037380000394100004243000006
:10111000444500004630000078000000436F0000A6
:10112000756C0000646E000027740000206B0000E6
:101130006565000070200000757000000000000070
:101140005350000049310000000000000029000059
:10115000002000005700000020520000004900005D
:1011600032430000310000003A200000000000007F
:101170002E00000031570000303100000000000058
:10118000314100004C530000004200005076000046
:1011900033000000080800000808000008000000F4
:1011A00000000000204800007A000000000000005D
:1011B00042420000494F000031000000524100004F
:1011C00057310000000000004F4300004431000090
:1011D00000000000000000000000000029000000E6
:1011E0000000000000000000EC874700889FBE0060
:1011F0008A9FBE008C9FBE008E1F78000000EB000F
:101200001064880000648800A04088002064880082
:101210000001780063C820000042EB0005022000B6
:101220004510DD00030040008000EB00045878000A
:101230008100E800858F5000FCFF3A000201E800C1
:10124000E50F5100F6FF3A000000EB00306988001E
:1012500080067800E0B79F00D0B79F00ACAE2000BA
:10126000A1408000E00220000089B9002095200004
:10127000000041005057020000000000A181200042
:1012800000202000110060000400320071002000E6
:10129000E05620009A7302000000000060722800EF
:1012A00050570200000000000001EB00C2B79F0091
:1012B00001003700CEB79F00306980000000E000D9
:1012C000440032000000E900306988004500DD007C
:1012D00061C82000E0C078000104E0001300320083
:1012E0000004EB0009B820006AC8200000648000F8
:1012F00001F07C0001407800DC5A02000000000090
:10130000006480000000E8000804E800F00FB2006C
:1013100000648800306980004500DD00080040005E
:10132000E0407D000104E000F0FF3A000000EB0027
:1013300030698800270037009C40780064C0600056
:10134000240032004A8120001A007800E9022000BF
:101350000980B9007A004000C892200060007C003B
:10136000000001000000E0001A0032001A007800BE
:101370000980B9006002B000080040005057020028
:1013800000000000607228005057020000000000BA
:101390001064800001648000810F50000D00320055
:1013A00000047800808F50000A00320009B8200045
:1013B00068C07C00DC5A02000000000008007800D1
:1013C000F00FB2000004E80000648000800F5400B9
:1013D000F7FF3A00425A0200000000000004E0005B
:1013E000D5FF3200F85A0200000000000004E000BF
:1013F00003003200005B020000000000AEFF370077
:10140000C85A020000000000004578000080FB0080
:1014100001002000F2072000820F5000E08F5800EA
:1014200081023E0000600100770237003F02370072
:10143000130137007C023700BD0037004E02370031
:101440002501370078023700770037007602370031
:101450005C0237007402370073023700590237000C
:101460009901370070023700290137006E023700FA
:101470006D0237006C0237006B0237006A023700DA
:1014800069023700680237006702370066023700DA
:1014900065023700D300370063023700620237006D
:1014A00061023700600237005F0237005E023700DA
:1014B0005D0237005C0237005B0237005A023700DA
:1014C00059023700580237005702370056023700DA
:1014D00055023700540237005302370052023700DA
:1014E00051023700500237004F0237004E023700DA
:1014F0004D0237004C0237004B0237004A023700DA
:1015000049023700480237004702370046023700D9
:1015100045023700440237004302370042023700D9
:1015200041023700400237003F0237003E023700D9
:101530003D0237003C0237003B0237003A023700D9
:1015400039023700380237003702370036023700D9
:1015500035023700340237003302370032023700D9
:1015600031023700300237002F0237002E023700D9
:101570002D0237002C0237002B0237002A023700D9
:1015800029023700280237002702370026023700D9
:1015900025023700240237002302370022023700D9
:1015A00021023700200237001F0237001E023700D9
:1015B0001D0237001C0237001B0237001A023700D9
:1015C00019023700180237001702370016023700D9
:1015D00015023700140237001302370012023700D9
:1015E00011023700100237000F0237000E023700D9
:1015F0000D0237000C0237000B0237000A023700D9
:1016000009023700080237000702370006023700D8
:1016100005023700040237000302370002023700D8
:10162000010237004200370010648000808F5600AE
:101630003B00320000648000808F56000B003A00AF
:101640000D00E90080067800FD0FB2000D648800EF
:101650000040EB0003B8200080F67900807228007B
:10166000505702000000000013FF37000D00E90092
:1016700080067800FD0FB200C072280050570200AB
:10168000000000000D0178008D0078008004EB0060
:10169000006480008D0F5000140032008004EB00C5
:1016A0000AB820000204E80068407D0000717D0057
:1016B0000004E00003003200DC5A020000000000D9
:1016C0000300370000C2B300DC5A02000000000033
:1016D0008904E80008017800F20FB2008200780067
:1016E00000648000820F5000EEFF3A000100E90024
:1016F000F00FB20000648800007328005057020009
:1017000000000000094078002C5902000000000091
:10171000307328005057020000000000E6FE37003A
:1017200070C0B300DC5A020000000000E2FE370087
:1017300000648000808F5600260032008D00780003
:101740000D0178000005EB008D0F500014003200F1
:101750000005EB0009B820000104E80068C07C0027
:1017600080F07C000004E00003003200DC5A02003C
:10177000000000000300370000C2B300DC5A020082
:10178000000000000A05E80088007800F10FB200B0
:101790000101780000648000810F5000EEFF3A00E4
:1017A0000200E900F00FB200006488000073280016
:1017B00050570200000000000A4078002C59020037
:1017C00000000000307328005057020000000000A5
:1017D000B9FE370070C0B300DC5A02000000000000
:1017E000B5FE3700C85A020000000000B1C5B300C2
:1017F000814F5000B0FE3A00C85A020000000000BD
:101800008040780010C4B30080CF50004000320008
:1018100007003E007040500080CF50000C003200A6
:101820006340400080CF5000A3FE3A000E00370016
:1018300030C4B30080CF500027003200A20039002E
:101840000040E80080CF50009BFE3A000C003700BB
:10185000C85A020000000000E1C7B300814F5000E9
:1018600095FE3A0031013700C85A0200000000001E
:10187000E1C7B300814F50008FFE3A003E013700B0
:101880005FB09700E40F5000050034007666020058
:10189000000000008000EB00D1B79F0086FE3700FB
:1018A00010648000808F5600070032000D00E900B0
:1018B00080067800FD0FB200C07228005057020069
:1018C000000000007CFE370070C0B300DC5A02004C
:1018D0000000000078FE370000648000808F560012
:1018E000070032000D00E80080067800FD0FB2000E
:1018F0005073280050570200000000006EFE3700B1
:1019000070C0B300DC5A0200000000006AFE37001D
:10191000146480000400E90000047800F80FB200AD
:101920000805780001648000810F540062003200D5
:101930008002EB0003B8200068C079000004E000DA
:1019400057003A000800E90000017800F20FB200E9
:1019500062C079000004E000510032008502E80016
:10196000CFB19700858F51004D0031008301E80011
:10197000C3B79F00810F52000A00320003B8200055
:101980008042EB00F60F200085F079000100E900AD
:1019900086006000810F5200FBFF3A00016488005E
:1019A00085F0790001648000828F5000AB053A0019
:1019B0000D00370003B8200062C079000004E00089
:1019C00004003A000200E800F00FB200E0B79F0008
:1019D000050037000200E90000017800F20FB200B4
:1019E000828F5000F3FF3A00907328005057020096
:1019F00000000000A1408000E00220000089B90042
:101A00002095200000004100505702000000000017
:101A1000A18120000020200011006000040032009D
:101A200071002000E05620009A73020000000000C0
:101A30006072280050570200000000006FB097004D
:101A4000880F50000F003200800478000BB820008F
:101A5000FD0F200069C07D00DC5A0200000000007C
:101A60000064800069F07D000000E8000D00600067
:101A7000006488000900E8008D046000890F5400AC
:101A8000F4FF3A000D6480000040EB0002B8200033
:101A9000807679008A8F560007FE3A0006003700EC
:101AA0000800E90000047800F80FB200080578008B
:101AB000888F50009FFF3A0070C0B300DC5A0200CC
:101AC00000000000FCFD3700146480000400E90001
:101AD00080047800F90FB2000905780001648000E5
:101AE000818F5400620032000007EB0003B8200031
:101AF00069C079000004E00057003A000900E900DD
:101B000000017800F20FB20062C079000004E0002A
:101B1000510032000E07E800CFB197000300E90042
:101B20008E0F50004C003A00810F52000A00320024
:101B300003B820008042EB00F60F200085F079000A
:101B40000100E90086006000810F5200FBFF3A00AF
:101B50000164880085F0790001648000828F500064
:101B600043053A000D00370003B8200062C0790039
:101B70000004E00004003A000200E800F00FB200A8
:101B8000E0B79F00050037000200E900000178007F
:101B9000F20FB200828F5000F3FF3A0090732800DA
:101BA0005057020000000000A1408000E002200029
:101BB0000089B90020952000000041005057020024
:101BC00000000000A1812000002020001100600022
:101BD0000400320071002000E05620009A730200D9
:101BE0000000000060722800505702000000000052
:101BF0006FB09700890F50000F003200000478008A
:101C00000BB82000FD0F200068C07D00DC5A0200E8
:101C1000000000000064800068F07D000000E80023
:101C20000D006000006488000800E8000D046000FA
:101C3000890F5400F4FF3A000D6480000040EB006F
:101C400002B82000807679008A8F560099FD3A000C
:101C5000CEB79F00060037000900E9008004780035
:101C6000F90FB20009057800898F50009FFF3A00F4
:101C70004FB09700E10F500028003A009073280001
:101C80005057020000000000A1408000E002200048
:101C90000089B90020952000000041005057020043
:101CA00000000000A1812000002020001100600041
:101CB0000400320071002000E05620009A730200F8
:101CC0000000000060722800505702000000000071
:101CD0000D64800011648000818F5600090032007D
:101CE00002B820008041EB00F40F200083767900D9
:101CF0000D00E90084066000818F5600FBFF3A006A
:101D00000D6488000040EB0001B8200080F67800E8
:101D10000001EB00C2B79F0067FD370070C0B30041
:101D2000DC5A02000000000063FD370018648000E8
:101D3000888F56000C0032000073280050570200B4
:101D40000000000008805600F00FB2002C5902007D
:101D5000000000003073280050570200000000000F
:101D60001D64800054FD370070C0B300DC5A0200CF
:101D70000000000050FD370008648000888F560086
:101D80000C003200007328005057020000000000D1
:101D90000D005400F00FB2002C59020000000000AA
:101DA000F073280050570200000000000D6480000E
:101DB00041FD370070C0B300DC5A02000000000093
:101DC0003DFD3700006480008040EB0003B8200038
:101DD00001F079000000E80080067800FD0FB200F5
:101DE0000D6488001074280068570200000000008D
:101DF00000648000F0B79F001E6480000000EB00CC
:101E00002064880053003700DFB097008100E800AD
:101E1000D1B79F00F48F500027FD3A00705B02009D
:101E20000000000024FD3700086480000800E8007E
:101E3000F90F20000900600011648000810F50003C
:101E400040003200FF4F55003E003600E0C7B300AF
:101E5000804F55003B003E008D0F54000C003A00AF
:101E60000A407800DC5A0200000000000064800094
:101E700002B820000A7079000000E80089066000BE
:101E80000D6488000040EB00807679000AFD370081
:101E90000073280050570200000000000D0054009D
:101EA000F80F2000080060002C590200000000001C
:101EB000F073280050570200000000000964800001
:101EC0000D00E90088056000898F55001000320080
:101ED00008B820000900E80069707C0069407C00B7
:101EE0000004E00005003200DC5A0200000000009F
:101EF0002074280050570200000000000900E9008B
:101F000080047800F90FB200898F5500F1FF3A0084
:101F10000A407800DC5A02000000000000B82000EF
:101F20008A7678000D00E800F10F2000810660003D
:101F3000006480000000E800010060000064880088
:101F4000DDFC370070C0B300DC5A02000000000066
:101F5000D9FC37001264800001B8200062C078000C
:101F60000080FB0001002000E3072000830F5000E9
:101F7000E08F580010043E0000600100100437009C
:101F80000D0437000C0437000B0437000A04370037
:101F90000904370008043700070437000604370037
:101FA0000504370006043700030437000204370035
:101FB0000304370000043700FF033700FE03370037
:101FC000FD033700FC033700FB033700FA0337003B
:101FD000F9033700F8033700F7033700F60337003B
:101FE000F5033700F4033700F3033700F20337003B
:101FF000F1033700F0033700EF033700F003370039
:10200000D00337005F023700120137001B01370091
:10201000BC013700AA013700E70337003C02370054
:10202000E5033700E4033700E5033700E403370036
:10203000840337009B0337006A033700C20237006E
:10204000C1023700C0023700BF023700BE023700AE
:10205000BD023700BC023700BB023700BA023700AE
:10206000B9023700D4033700D3033700C10137006A
:10207000B8003700D00337003F0037002901370090
:102080001D013700CC03370061003700890137009C
:10209000C9033700C8033700C7033700C60337003A
:1020A000C5033700C4033700C3033700610037009E
:1020B000C1033700C0033700BF033700810037007A
:1020C000BD033700BC0337009F013700BA03370058
:1020D000B9033700B803370026013700B6033700CD
:1020E000B5033700B40337007802370049033700DF
:1020F00085023700790337005E033700AE033700EF
:10210000F2003700270037003A0037005B01370044
:10211000A9033700290037002B003700A803370038
:1021200018003700A4033700A30337004A00370024
:102130001A003700A00337001C0037004F0037009B
:102140009D033700E30237009B0337009A033700F3
:102150009903370017003700360137009603370020
:1021600095033700940337005F0237009100370072
:102170006D023700AA003700FE7302000000000065
:102180008F0337009F050700408120001000E0000A
:102190008B03320010060700890337009D040700F7
:1021A000870337002E070700850337000D07070058
:1021B000830337008D06070081033700E0540200D7
:1021C000000000007E033700408120001000E00086
:1021D00005003A00D1012000505A2000F47302009B
:1021E00000000000760337008E530200000000005C
:1021F00073033700C0CFB3001C4E600061012000A4
:10220000A0572000F4730200000000006C033700A8
:102210001C4078000014A1000004A000004E7800CB
:102220005101200000592000F4730200000000005A
:10223000630337001C34A000C1012000E07E2000B1
:102240009A73020000000000107428006857020012
:10225000000000005A0337001C34A100B101200027
:10226000307D20009A7302000000000010742800E6
:102270006857020000000000510337004081200031
:102280001000E00005003A00D1012000505A200063
:10229000F47302000000000049033700CB62A9007C
:1022A000C962A90051012000205C20009A7302003D
:1022B00000000000107428006857020000000000B1
:1022C0003F033700408120001000E00005003A0085
:1022D000D1012000505A2000F473020000000000D9
:1022E000370337009C40780070C0600004003A005B
:1022F00021022000F0E92000F47302000000000039
:10230000C962A800CB62A90041012000705D2000D5
:102310009A73020000000000107428006857020041
:102320000000000021E3A800B0C0B3001672020054
:1023300000000000F1042000810F500003003E0067
:1023400070742800685702000000000021E3A90013
:102350001B0337000200E800F00FB2001064880091
:102360001C040700500307000004780072590200A3
:1023700000000000A0762800505702000000000076
:10238000084078002C59020000000000A0762800C8
:1023900050570200000000000840780088570200F3
:1023A00000000000107428006857020000000000C0
:1023B000030337000200E800F00FB2001064880049
:1023C00004040700380307000080FB00727302005A
:1023D00000000000000478007259020000000000B4
:1023E000A076280050570200000000000840780046
:1023F0002C59020000000000A0762800505702006F
:10240000000000000840780088570200000000002B
:10241000107428006857020000000000E80237002E
:10242000408120001000E00005003A0011C0B30018
:10243000014078004C6B020000000000E002370011
:10244000A1012000B05E2000F47302000000000033
:10245000DB0237005100200050602000F4730200BE
:10246000000000003A5A0200000000000004E000F2
:10247000FCFF32000000FE00D10237008A74020027
:10248000000000000000E000CD023200A1002000AA
:10249000A0602000F473020000000000400620004D
:1024A0002073020000000000D8710200000000004C
:1024B0003A5A0200000000000004E000FCFF320075
:1024C00081BF2A0001400100BD02370093030700CD
:1024D000800478000000E000B90232000004EB0044
:1024E00004560200000000000804E800888F540031
:1024F000B3023200FAFF3700880307008004780037
:102500000000E000AE0232000004EB00E8550200DB
:10251000000000000804E800888F5400A802320080
:10252000FAFF37007D030700800478000000E00018
:10253000A30232000004EB00610120004061200092
:102540009A73020000000000205602000000000004
:102550004057020000000000107428006857020075
:10256000000000000804E800888F54009402320044
:10257000F1FF3700408120001000E00005003A0024
:10258000D1012000505A2000F47302000000000026
:102590008B023700C002A900C202A80021E3A800F4
:1025A000200020002073020000000000A0C0B30043
:1025B0001672020000000000011B2000810F500075
:1025C0000E00360090C0B30016720200000000003A
:1025D000712B2000810F50000800360011012000EF
:1025E000A06220009A73020000000000107428000E
:1025F00068570200000000000C003700C002A9006C
:10260000C202A900E076280068570200000000001E
:1026100021012000B06320009A7302000000000036
:1026200010742800685702000000000021E3A90090
:1026300063023700408120001000E00005003A00EE
:10264000D1012000505A2000F47302000000000065
:102650005B023700C002A900C202A90021012000CC
:10266000B06320009A73020000000000107428007C
:10267000685702000000000051023700F1002000FE
:10268000C03620009A730200000000002872020089
:102690000000000011002000B03720009A730200F3
:1026A00000000000107428006857020000000000BD
:1026B000430237003672020000000000400237007B
:1026C00016030700000478006100200090652000D8
:1026D0009A7302000000000008007800E25802002F
:1026E0000000000021002000F0652000F4730200CB
:1026F00000000000080078004473020000000000A1
:102700002F02370005030700000478006100200055
:10271000906520009A730200000000000800780015
:10272000E2580200000000002100200030EE2000EE
:10273000F47302000000000008007800207302001B
:10274000000000001E023700408120001000E00061
:1027500005003A00D1012000505A2000F473020015
:10276000000000001602370046560200000000007C
:102770001302370011002000216488000200E800E5
:102780008081FB0000B82000634078000004E00076
:102790001300320001027800E6C3B300F70F2000F7
:1027A00005B82000864F500001003A000002EB00FF
:1027B0008100E800010041000700600060C07A006D
:1027C0000004E000F7FF3A002464880020022000A3
:1027D000808F500002003400100020002064880028
:1027E000296480000900E000F5013A0013648800C4
:1027F0002D0207000004780012648000F30F20000F
:102800008300610000B82000E1407800D0C3B3002D
:1028100080CF50001E003A000802E900E40F520089
:1028200018003E000200E800830160001364880085
:10283000C520DD0060C820008080400009007800CD
:102840000041EB0005022000825878000000E800FB
:10285000850F50000B023200FBFF370082587800D2
:102860000300E8008081FB0000B82000634178008D
:10287000E0C3B300804F5100F8FF3A0013648800B2
:10288000CF0137001000200020648800CC01370001
:102890000800E00013003A0069C82000180020007A
:1028A000084078002C59020000000000E078280061
:1028B0005057020000000000090078005057020045
:1028C000000000006072280068570200000000004D
:1028D0000804E8000902B000E60F5400B801320015
:1028E000EFFF37000800E900E40F500005003E004C
:1028F0001074280068570200000000003869880042
:10290000AF0137001000200020648800AC013700C0
:102910000200E800F80F2000080060001064880042
:10292000E101070080047800AA020700106480001B
:102930000800600001B82000E0C0780090C2B30039
:1029400080CF50000C003A00A0408000E20220003E
:102950000280B9007C004000C2922000E0007900B3
:102960000900780001000100107428006857020077
:102970000000000092013700100020002064880051
:102980008F01370013002000236488000200E80054
:102990000080FB0001B8200060C078000004E00067
:1029A0000E0032008280E8000301780025C2B300E7
:1029B000F30F200004B82000854F500001003A00BA
:1029C0000001EB000380600060407A008100E800B5
:1029D0000004E000F8FF3A002264880020648000D0
:1029E0000000E00076013A0071002000106620002F
:1029F0009A7302000000000020C2B300DC5A0200FB
:102A000000000000106480000000E80010648800EE
:102A10000081FB0000B82000E240780020C2B30033
:102A200080CF50002100320008B8200012648800D6
:102A300001407800DC5A02000000000010648000B1
:102A400060407C008001FB00A0AE200010407800B8
:102A500068406000040032000300780072730200D6
:102A60000000000080017800A0408000E202200009
:102A70000280B90068004000C2922000E0007900A6
:102A80000300780001000100106480000000E800ED
:102A90001064880000017800F20FB200E2407C0070
:102AA00020C2B30080CF5000E0FF3A0012648800DB
:102AB00020C2B300DC5A020000000000107428009D
:102AC00068570200000000003D013700A040800070
:102AD000E20220000280B900C29220006200780069
:102AE0000000010036013700A0408000E202200013
:102AF0000280B9000080E800C292200060007900E6
:102B0000000001002E013700A0408000E2022000FA
:102B10000280B90064004000C29220006000790089
:102B20000000010026013700A0408000E2022000E2
:102B30000280B90066004000C29220006000790067
:102B4000000001001E013700710020001066200007
:102B50009A7302000000000053010700800478000F
:102B6000106480000000E9000080FB001064880011
:102B7000EA01070080BF9F00FF0107008000780086
:102B80000000E0000900320090AD2000014878000C
:102B9000E88F500003003400A0AE20001054A000C5
:102BA00002003700A0AE20001054A1008005EB0009
:102BB0004100370009007800947202000000000014
:102BC00003C2B300A2AE200012C0610005003A00AB
:102BD00081C0B30090AD200090CF100005003A00F6
:102BE0000B00370003C1B30092AD200092CF11005B
:102BF00007003200B0C3B300DC5A0200000000003E
:102C000091AD2000114078002C5902000000000016
:102C1000A2AE20001241780068406100040032003A
:102C20000900780072730200000000008004780040
:102C3000A0408000E20220000280B900680040004D
:102C4000C2922000E0007900090078000100010034
:102C50000004780000C2B300DC5A0200000000004B
:102C6000AAAE200003C4B3001AC0610011003200F4
:102C700061002000806620009A73020000000000BE
:102C80001A457800684065000400320008007800AA
:102C90007273020000000000000478000800780051
:102CA000947202000000000000C2B300DC5A02006F
:102CB000000000008B05E8000FB89700808F5500DA
:102CC000BCFF3A00107428006857020000000000A2
:102CD000BB00370061002000806620009A7302006C
:102CE000000000008D01070000057800A201070028
:102CF000800078000000E0000900320090AD200064
:102D000001487800E88F500003003400A0AE200096
:102D10001054A00002003700A0AE20001054A10003
:102D20000A00E0002B0032000004EB00ABAE2000F4
:102D300099AD2000A0408000E20220000280B9008E
:102D40006A004000C292200060007900000001008B
:102D5000800078001B417800684061000400320068
:102D6000010078007273020000000000800078000B
:102D700001007800947202000000000003C2B3005A
:102D80001BC0610004003A0080C0B300994F1000DE
:102D900004003A000900370001C1B30099CF1000C8
:102DA00006003200B0C3B300DC5A0200000000008D
:102DB000194078002C5902000000000000C2B30046
:102DC000DC5A0200000000000804E800880F5500EB
:102DD000D8FF3A0010742800685702000000000075
:102DE0007700370081002000E0662000F4730200C5
:102DF00000000000A0408000E20220000280B90034
:102E00006C004000C29220006000790000000100C8
:102E10006B0037008100200060672000F47302001F
:102E200000000000A0408000E20220000280B90003
:102E30006E004000C2922000600079000000010096
:102E40005F003700E1002000E0672000F47302001B
:102E500000000000A0408000E20220000280B900D3
:102E600070004000C2922000600079000000010064
:102E700053003700E1002000C0682000F473020016
:102E800000000000A0408000E20220000280B900A3
:102E900072004000C2922000600079000000010032
:102EA00047003700C1002000D06420009A73020060
:102EB00000000000A0408000E20220000280B90073
:102EC00074004000C2922000600079000000010000
:102ED0004057020000000000390037000F010700D2
:102EE00000047800D1002000A06A20009A7302003C
:102EF000000000000800780094720200000000004A
:102F00000800E0000B0032008004EB00EA02200021
:102F1000CB922000A04080000A80B90076004000DB
:102F200060807D00000001008904E800890F5400E2
:102F3000F8FF3A00107428006857020000000000F3
:102F40001F003700F500070080047800A100200072
:102F5000706B20009A730200000000000900E0007E
:102F6000100032000004EB00EA022000CB922000A7
:102F7000A04080000A80B9007800400060807D0099
:102F800000000100405702000000000000C2B30032
:102F9000DC5A0200000000000804E800888F54009A
:102FA000F3FF3A0001012000A0692000F473020041
:102FB000000000000200370010002000206488009C
:102FC000106480000000E8000080FB0010648800AE
:102FD000206480000000E00002003A000001780058
:102FE0001400370051012000106C20009A73020079
:102FF0000000000010648000800F570004003100C2
:103000000E4050002C590200000000000300370061
:103010000E4050002C590200000000000000EB00A0
:103020002064880010742800685702000000000027
:10303000120020001164800000648000808F500026
:10304000020032000200E000C2FB32007FB19700B4
:10305000126488000264880081F8370000B82000FC
:10306000624078000004E00056FA320059FA370056
:1030700000B82000624078000004E000BEFA320090
:10308000C1FA370000B8200063417800E0C3B30004
:10309000804F5100CAFF3200C520DD0060C820000B
:1030A00080804000EDFD3700881F780015648000A7
:1030B000F40F20000480620003B82000E0C0790013
:1030C000F0CCB30000C04000E84F50001A003E00B2
:1030D0000100FB0001FD2F00010140000500E80098
:1030E0000400600060C279008140420016002000A8
:1030F000E9CF500077003E001600200001FD2F00B0
:10310000F80F200007B820006A11B9000400FB0086
:1031100002004000010140000603E8000680420072
:103120000800600060C27B0001404200E94F50008F
:1031300068003E00F4FF370000C3B30080CF5000AA
:1031400060003A000500E8000080FB0001B82000A4
:1031500060C2780020C6B300804F52006100320088
:1031600020C4B300804F520012003A005D003700C7
:10317000260020000001EB0003FD2F00F70F2000C8
:1031800004B82000020041008100FB000100400063
:10319000030140000603E8000680420007006000CB
:1031A000E0407A0003C04000E14F500049003E007B
:1031B000F4FF370080C7B300804F52001600320082
:1031C00080C5B300804F520026003A00120037003D
:1031D0004411DD00E9CF510005003E000100FB0075
:1031E0000000410001FD2F000101400008003700F0
:1031F000014078000054A00001B8200000F27800DF
:103200000000FB000000410091FA2F000101400086
:103210000603E80002003700260020000001EB0052
:10322000068042000082FB0000B82000E4407800E5
:1032300000CDB30080C14000E9CF5100E4FF36006B
:103240007140500000C04000E54F5000E0FF3600E4
:10325000F0C9B30000C04000E54F5000DCFF36006D
:103260001C00370000CDB3000040420016002000D3
:103270000001EB00E94F500016003E008400FB0007
:1032800000FD2F000081400080007800F80F200032
:1032900007B820006A11B9000400FB0002004000DA
:1032A000010140000603E80005004300080060003B
:1032B00060C27B0001404200E94F500005003E0023
:1032C000F4FF370010002000206488000001EB00AC
:1032D0000F003700068042000080FB001064880069
:1032E0000B0037000580E8000080FB0001B82000DB
:1032F000E0C0780000CDB30000C0400026002000F0
:103300000001EB00E14F5000F2FF3E0098FF370054
:10331000020078004F04780000000600881F780043
:10332000126480000200E8000080FB0001B8200069
:10333000E0C0780013002000A0C3B30080CF50008D
:103340000A003A000280E800F80F20000800600040
:103350001064880054FF070080017800106480002A
:103360000000E90008006000106488000300780095
:103370004F04780000000600881F78001264800067
:103380000200E8000080FB0001B82000E0C07800E7
:103390008001EB00B0C3B30080CF50000A003A00B8
:1033A0000280E800F80F2000080060001064880028
:1033B0003DFF070080017800106480000000E900F4
:1033C0000800600010648800030078004F04780053
:1033D000000006001264800000B82000E24078007F
:1033E00000C2B30080CF500009003A00F40F200063
:1033F00003B82000804078000200E800040160006B
:1034000062C07900814F5000FBFF320012648800D7
:1034100000000600889FBE008A9FBE008C1F7800B7
:10342000106480000000E8000080FB001064880049
:10343000E8FF07001CFF07000000E0003C003A0026
:1034400018002000EB022000CA92200008407800FB
:103450002C5902000000000020792800505702007B
:10346000000000000BC0B900680050000A004000D6
:1034700068570200000000000804E800E90F54004B
:10348000F2FF3A0071012000606D2000F473020029
:10349000000000000000EB00206488001300200002
:1034A00082002000830078000300780046000700B7
:1034B0000006E9000000E800E10F500005003E00B2
:1034C000E1002000D06E2000F47302000000000034
:1034D000350037004B8120001B007800E8022000F7
:1034E0000880B9000002B000CA92200060007D0090
:1034F00000000100D8710200000000008C0D78006F
:1035000008E4B9007E04440068007D00000001006A
:103510000C00E00001003200C222A800510020008F
:1035200050572000F4730200000000001E00370016
:103530000006E900E70F560017003C004B81200011
:103540001B007800E80220000880B9000002B000EB
:10355000CA92200060007D0000000100D8710200C6
:10356000000000008C0D780008E4B9007E044400DF
:1035700068007D00000001000C00E0000100320046
:10358000C222A8005100200050572000F47302000E
:10359000000000000400370051012000C07220002C
:1035A000F473020000000000006480000000E900E5
:1035B0000080FB00106488004F0678004F05BE00B5
:1035C0004F04BE0000000600E8874700889FBE0049
:1035D0008A9FBE008C9FBE008E1F78000005BE0033
:1035E00082067800030778005079280050570200BF
:1035F000000000000A00E00004003D00907928006F
:103600005057020000000000030037000A40780015
:103610002C59020000000000B07928005057020029
:10362000000000008004EB00090678003600370037
:103630000900E000050032008904E90080722800DA
:1036400050570200000000002F0037000C00E0007F
:10365000060032008072280050570200000000006F
:103660008004EB00090678002700370070C0B30023
:10367000DC5A0200000000008004EB00220037004A
:103680000900E00005003A00D0C2B300DC5A020095
:10369000000000001C0020001B00370070C0B300B9
:1036A000DC5A020000000000170037000E00E000A6
:1036B00046003A0000CDB30000404400E94F5000FE
:1036C0000E003E00E38F54000500340070C0B300CC
:1036D000DC5A020000000000490020000A00370008
:1036E00008407800DC5A020000000000748054009A
:1036F00008F07F008904E8000300370070C0B300C1
:10370000DC5A020000000000C85A0200000000005D
:1037100000447800ED4F50002E00320005003C00C0
:10372000E84F5000C2FF3200EA4F5000E1FF3A007C
:1037300028003700D0C2B300804F5400D0FF3200C1
:1037400080C7B300804F5400DAFF3A00D7FF37003C
:103750000901E9000000EB000D0033000000EB0060
:103760008000780005FD2F000202E8006A01B90020
:103770007483570066C078000000FB000200400020
:10378000050040008100E800848F5000F7FF3A00F8
:10379000808F550008003C00808F560006003500E1
:1037A0000C00E00002003A00000578000E0037002F
:1037B0000005EA000C003700B101200080EC200079
:1037C000F47302000000000087FF37000085EB0063
:1037D0000500370010742800685702000000000040
:1037E0000900E000DAFF3A000A0078004F0778008D
:1037F0004F06BE004F05BE004F04BE008F00B10053
:1038000000000600881F7800E07928005057020069
:1038100000000000E0C2B300DC5A0200000000001B
:10382000A081200010407800DC5A02000000000057
:1038300061812000F0442000910F100003003A0045
:10384000C07A2800505702000000000010742800C1
:103850006857020000000000307C2800505702002A
:1038600000000000D1002000A08020009A73020018
:1038700000000000A1BF2A000000EB00025A020075
:1038800000000000000478004800DE002C5902000F
:1038900000000000E0C2B300DC5A0200000000009B
:1038A000084078002C590200000000001074280025
:1038B0006857020000000000610020003076200000
:1038C0009A73020000000000688120001800780050
:1038D000AE590200000000007100200010EC200032
:1038E0009A73020000000000C0408000AE59020040
:1038F00000000000E07D280050570200000000009A
:10390000F0442000980F100004003A00B07E280018
:10391000505702000000000003003700E07E28003E
:103920005057020000000000C14080002004230026
:10393000808F50001000320004003E003000230051
:10394000808F500018003A00070037003004230031
:10395000808F50000C00320063004000808F5000C8
:1039600011003A000C003700107F28005057020069
:10397000000000000F003700407F28005057020071
:10398000000000000B003700707F28005057020035
:103990000000000007003700A07F280050570200F9
:1039A0000000000003003700D07F280050570200BD
:1039B000000000001080280068570200000000008E
:1039C000E101200090762000F47302000000000066
:1039D0004F047800000006005100200050922000A3
:1039E0009A73020000000000C1BF2A000000EB0033
:1039F000025A020000000000AE5902000000000060
:103A000061002000A09220009A73020000000000D4
:103A1000E1BF2A000000EB00025A02000000000093
:103A2000AE59020000000000107428006857020020
:103A300000000000C100200070782000F473020034
:103A40000000000069000700C2C2BF000008A30018
:103A50000500320011012000A06220009A730200CC
:103A6000000000000400370021012000B0632000A6
:103A70009A73020000000000C0C2B300DC5A0200CA
:103A80000000000000C2B300DC5A02000000000089
:103A9000CBC2BF000038A300050032004101200066
:103AA000705D20009A7302000000000004003700DF
:103AB00051012000205C20009A73020000000000E9
:103AC000C0C2B300DC5A02000000000000C2B30014
:103AD000DC5A020000000000A0AE20001040780078
:103AE0007040600005003200210220003079200083
:103AF000F47302000000000004003700E101200020
:103B0000507B2000F473020000000000A0AE2000F3
:103B1000104078006840600005003A00B1012000C4
:103B2000307D20009A73020000000000040037007E
:103B3000C1012000E07E20009A7302000000000016
:103B4000C0C2B300DC5A02000000000000C2B30093
:103B5000DC5A020000000000B1012000B01A210070
:103B60009A7302000000000090AD20001040780021
:103B70002C59020000000000107428006857020051
:103B800000000000A0AE20001040780063406000FC
:103B9000E14F500005003A0051012000005920007B
:103BA000F4730200000000000400370061012000EF
:103BB000A0572000F473020000000000A040800025
:103BC000E20220000280B9004002B000C292200050
:103BD0006000790000000100C10020007078200022
:103BE000F47302000000000000000600A1002000A5
:103BF00040072100F473020000000000610420006F
:103C0000C00C2100F473020000000000A10120009C
:103C1000E00721009A73020000000000A04080002D
:103C2000E20220000280B9002002B000C29220000F
:103C30006000790000000100A1002000800921003F
:103C40009A73020000000000004020004F000700AF
:103C5000001020004D000700002020004B0007004E
:103C6000000420004900070000082000470007006A
:103C70001074280068570200000000004100200076
:103C8000201121009A7302000000000021E3A80027
:103C9000A0C0B3001672020000000000D859020054
:103CA0000000000011002000B03720009A730200CD
:103CB0000000000090C0B300DC5A020000000000C9
:103CC00090C0B3001672020000000000D859020034
:103CD0000000000011002000B03720009A7302009D
:103CE0000000000090C0B300DC5A02000000000099
:103CF000C0C0B3001672020000000000D8590200D4
:103D00000000000011002000B03720009A7302006C
:103D10000000000090C0B300DC5A02000000000068
:103D2000B0C0B3001672020000000000D8590200B3
:103D30000000000011002000B03720009A7302003C
:103D40000000000090C0B300DC5A02000000000038
:103D500021E3A90000402000170007000010200008
:103D600015000700002020001300070000042000B9
:103D700011000700000820000F0007001074280041
:103D80006857020000000000000006004116800095
:103D9000808060000400320030802800505702000C
:103DA0000000000003003700608028005057020028
:103DB00000000000000006005116800080806000B6
:103DC00004003200908028005057020000000000DC
:103DD00003003700C0802800505702000000000098
:103DE00000000600881F7800106480000000E800D2
:103DF0000080FB001064880076FD0700AAFC070025
:103E00000000E900E30F500002003E0090408800EF
:103E10000D0037000004EB00286488002102200018
:103E200070812000F4730200000000008801780017
:103E3000420020001100200010002000E2FD0700D9
:103E40000000E900904088002101200090832000BC
:103E5000F4730200000000004F0478000000060028
:103E6000881F7800106480000000E8000080FB00DC
:103E70001064880057FD07008BFC07008040E900B4
:103E8000E9CF500003003E00008120000148780087
:103E90000D0037000004EB0028648800D1082000E2
:103EA00060872000F47302000000000088017800A1
:103EB000A20020001100200090002000C2FD070099
:103EC000018120008048E9000044EB0000812000CF
:103ED00091C0B30090CF100010003A003DFD0700E4
:103EE00071FC0700004478000004E0000B003A0079
:103EF0000004EB0028648800F08028006857020066
:103F00000000000088017800F2FF27008800780098
:103F100020022000ACFD0700004478004101200091
:103F200030902000F4730200000000001101200016
:103F3000A0192100F4730200000000003A5A0200A8
:103F4000000000000004E000FCFF320000812000BF
:103F500091C0B30090CF100003003A0008407800F1
:103F6000F25A020000000000185A0200000000008F
:103F700008C2B300C85A020000000000884F500079
:103F8000FCFF3A004F047800000006005752490039
:103F900054452000424954003A2020002A6E650012
:103FA00078742000636C6F00636B2000285E29002A
:103FB000207769006C6C20007573650020746800C0
:103FC0006973200076616C0075654E006F20640097
:103FD0006576690063652C002074720079202800E2
:103FE000414C4100524D29002053450041524300AD
:103FF00048206D00616372006F2066006972730073
:104000007441440044524500535320004D41430045
:10401000524F200020302E004D616300726F20004F
:104020006D656E00754D610063726F002020200089
:10403000202031005749520045206100646472001D
:10404000657373000D0A200020202A0031574900B3
:1040500052452000524F4D0020434F004D4D41002E
:104060004E4420004D414300524F73003A0D0A0068
:10407000203531002E52450041442000524F4D0062
:10408000202830007833330029202A00666F720020
:10409000207369006E676C006520640065766900B6
:1040A00063652000627573000D0A200038352E000C
:1040B0004D41540043482000524F4D00202830000D
:1040C0007835350029202A00666F6C006C6F770008
:1040D0006564200062792000363462006974200033
:1040E0006164640072657300730D0A002032300051
:1040F000342E53004B49500020524F004D202800D1
:1041000030784300432920002A666F006C6C6F00F2
:10411000776564002062790020636F006D6D610037
:104120006E640D000A20320033362E00414C4100EF
:10413000524D200053454100524348002028300092
:1041400078454300290D0A0020323400302E5300F8
:104150004541520043482000524F4D002028300076
:104160007846300029414C0041524D002053450013
:10417000415243004820280030784500432953002D
:10418000454152004348200028307800463029003D
:10419000446576006963650020494400732061002E
:1041A0007265200061766100696C6100626C650077
:1041B00020627900204D410043524F002C207300B3
:1041C00065652000283029002E524500414420001A
:1041D000524F4D002028300078333300293A200018
:1041E0004D41540043482000524F4D0020283000DC
:1041F0007835350029534B0049502000524F4D006F
:10420000202830007843430029556E006B6E6F0004
:10421000776E20006D616300726F2C002074720055
:1042200079203F00206F720020283000292066008E
:104230006F72200068656C00704255005320520078
:10424000455345005420570061726E00696E670047
:104250003A202A0053686F00727420006F722000A9
:104260006E6F200070756C006C2D750070202A0038
:104270004E6F200064657600696365002064650008
:104280007465630074656400204453003138530042
:104290003230200048696700682050007265730062
:1042A0002044690067205400686572006D44530023
:1042B000313842003230200050726F0067205200C7
:1042C00065732000446967002054680065726D00C2
:1042D0004453310038323200204563006F6E2000B5
:1042E000446967002054680065726D0044533200D1
:1042F00034303400204563006F6E7200616D200021
:1043000074696D0065204300686970004453320091
:104310003433310020314B002045450050524F00CE
:104320004D556E006B6E6F00776E200064657600F1
:104330006963650050574D00206469007361620035
:104340006C656400314B48007A2D34002C3030000D
:10435000304B48007A205000574D4600726571007E
:1043600075656E0063792000696E20004B487A0005
:104370002050720065736300616C65003A50520012
:10438000323A44007574790020637900636C6500EB
:1043900020696E002025200050574D0020616300E9
:1043A0007469760065455200524F52003A20500021
:1043B000574D200061637400697665002C2067000A
:1043C00020746F0020646900736162006C654100B5
:1043D0005558200046726500717565006E6379005E
:1043E0003A20410055582000494E500055542F00A6
:1043F00048492D005A415500582048004947480077
:1044000041555800204C4F0057564F004C544D001A
:104410004554450052204D004F444500564F4C0036
:104420005441470045205000524F4200453A200079
:1044300056457200726F720028292000406C690096
:104440006E653A0020407000676D73007061630014
:10445000653A20006279740065732E00546F6F0016
:10446000206C6F006E67210053796E0074617800D4
:1044700020657200726F72004E6F2000454550003B
:10448000524F4D004572610073696E0067646F00A2
:104490006E655300617669006E672000746F2000BE
:1044A000736C6F00742049006E7661006C69640063
:1044B00020736C006F744C006F616400696E67005C
:1044C000206672006F6D2000736C6F0074204500D1
:1044D00052524F00523A2000636F6D006D616E00C2
:1044E00064206800617320006E6F200065666600BE
:1044F000656374002068650072654100434B4E009F
:1045000041434B0049324300205354004152540070
:10451000204249005449320043205300544F500078
:10452000204249005449320043206D006F64650009
:104530003A0D0A0020312E0020536F006674770078
:10454000617265000D0A2000322E20004861720061
:1045500064776100726553006574200073706500B4
:1045600065643A000D0A2000312E20007E354B0094
:10457000487A0D000A2032002E207E0035304B0094
:10458000487A0D000A2033002E207E0031303000A2
:104590004B487A000D0A2000342E20007E34300073
:1045A000304B48007A574100524E49004E473A007E
:1045B00020484100524457004152450020493200F2
:1045C0004320690073206200726F6B00656E2000EB
:1045D0006F6E200074686900732050004943210009
:1045E00020285200455620004133290053657400AD
:1045F00020737000656564003A0D0A0020312E00BA
:1046000020313000304B48007A0D0A0020322E0055
:1046100020343000304B48007A0D0A0020332E0041
:1046200020314D00487A490032432000286D6F0048
:1046300064207300706429003D28200020302E0083
:104640004D616300726F20006D656E00750D0A008C
:1046500020312E00376269007420610064647200AA
:10466000657373002073650061726300680D0A0052
:1046700020322E004932430020736E0069666600C6
:104680006572530065617200636869006E6720009F
:104690004932430020616400647265007373200036
:1046A0007370610063652E0020466F00756E6400B4
:1046B00020646500766963006573200061743A00C8
:1046C000536E6900666665007228420041534900D6
:1046D000432952006561640079612F00412F400039
:1046E00020636F006E7472006F6C73002041550080
:1046F00058207000696E61002F412F004020630038
:104700006F6E7400726F6C00732043005320700052
:10471000696E43006F6D6D00616E6400206E6F0006
:10472000742075007365640020696E002074680051
:10473000697320006D6F6400655075006C6C2D000E
:104740007570200072657300697374006F72730076
:10475000204F4600465075006C6C2D00757020008F
:1047600072657300697374006F727300204F4E009E
:1047700053656C00662D74006573740020696E00CB
:10478000204869005A206D006F646500206F6E003C
:104790006C7952004553450054424F004F544C0031
:1047A0004F4144004552410055582000494E5000A9
:1047B00055542F0048492D005A2C200052454100E5
:1047C000443A2000504F57004552200053555000A6
:1047D000504C4900455320004F4E50004F57450064
:1047E00052205300555050004C49450053204F0073
:1047F0004646440041544100205354004154450072
:104800003A204400454C410059207500735752002E
:10481000495445003A205200454144003A204300A3
:104820004C4F43004B2C200031434C004F434B0076
:104830002C2030004441540041204F00555450007A
:1048400055542C002031440041544100204F550064
:1048500054505500542C200030202A0070696E00FE
:1048600020697300206E6F0077204800695A43006A
:104870004C4F43004B20540049434B00533A200017
:10488000524541004420420049543A0020537900E7
:104890006E7461007820650072726F007220610092
:1048A000742063006861720020782E002065780013
:1048B0006974280077697400686F7500742063005C
:1048C00068616E00676529006E6F20006D6F64007F
:1048D0006520630068616E00676523003A204E0022
:1048E0006F2073006F66740077617200652072003C
:1048F0006573650074206F006E207600342C2000F4
:10490000757365002074680065207200657365002A
:1049100074206200757474006F6E2E004E6F6E000E
:1049200065786900737465006E74200070726F00A2
:10493000746F63006F6C2100782E20006578690029
:10494000740D0A00496E7600616C69006420630092
:10495000686F690063652C00207472007920610023
:10496000676169006E444500564944003A68740026
:1049700074703A002F2F6400616E670065726F00DB
:1049800075737000726F74006F74790070657300D6
:104990002E636F006D2A2D002D2D2D002D2D2D0045
:1049A0002D2D2D002A4F7000656E2000647261006D
:1049B000696E20006F757400707574007320280094
:1049C000483D4800692D5A002C204C003D474E00C0
:1049D00044294E006F726D00616C20006F75740089
:1049E0007075740073202800483D33002E33760024
:1049F0002C204C003D474E0044294D0053422000DE
:104A0000736574003A204D004F53540020736900C1
:104A100067206200697420006669720073744C003C
:104A200053422000736574003A204C004541530006
:104A30005420730069672000626974002066690071
:104A40007273740020426F006F746C006F616400B9
:104A500065722000762031002E20480045580D0058
:104A60000A2032002E20440045430D000A20330066
:104A70002E204200494E0D000A2034002E20520004
:104A800041574400697370006C61790020666F00C3
:104A9000726D610074207300657456006F6C740051
:104AA00061676500206D6F006E6974006F7273003E
:104AB0003A203500563A2000207C2000332E330067
:104AC000563A2000207C2000565055004C4C550092
:104AD000503A2000536574002073650072696100CC
:104AE0006C2070006F727400207370006565640044
:104AF0003A20280062707300290D0A0020312E0030
:104B000020333000300D0A0020322E0020313200D8
:104B100030300D000A2033002E20320034303000B7
:104B20000D0A2000342E200034383000300D0A00E9
:104B300020352E002039360030300D000A20360096
:104B40002E20310039323000300D0A0020372E007F
:104B500020333800343030000D0A2000382E200079
:104B60003537360030300D000A2039002E20310054
:104B70003135320030300D000A3130002E20420035
:104B80005247200072617700207661006C756500E5
:104B900041646A007573740020796F00757220009B
:104BA000746572006D696E00616C41007265200071
:104BB000796F75002073750072653F0020434600D1
:104BC00047313A002043460047323A00285C2D0026
:104BD0002F5F5C002D2928005C5F2F002D295300DA
:104BE000656C6500637420006F75740070757400E7
:104BF0002074790070653A000D0A2000312E2000E3
:104C00004F7065006E206400726169006E2028009C
:104C1000483D4800692D5A002C204C003D474E006D
:104C200044290D000A2032002E204E006F726D00C4
:104C3000616C200028483D00332E3300562C2000A4
:104C40004C3D47004E442900523257002028730043
:104C50007064200068697A00293D28002020300017
:104C60002E4D610063726F00206D65006E750D0042
:104C70000A2031002E4953004F37380031362D00BD
:104C80003320410054520D000A2032002E495300B7
:104C90004F37380031362D003320700061727300B9
:104CA00065206F006E6C790049534F002037380043
:104CB00031362D0033204100545220002852450047
:104CC00053455400206F6E0020435300290D0A0005
:104CD000524553004554200048494700482C2000C5
:104CE000434C4F00434B2000544943004B2C2000C1
:104CF00052455300455420004C4F570049534F0034
:104D00002037380031362D003320720065706C007A
:104D10007920280075736500732063007572720036
:104D2000656E7400204C530042207300657474005B
:104D3000696E6700293A200050726F00746F63003B
:104D40006F6C3A0020736500726961006C3320005B
:104D500077697200653220007769720065524600FB
:104D600055756E006B6E6F00776E52006561640062
:104D70002074790070653A0020746F0020656E0021
:104D80006476610072696100626C6500206C650088
:104D90006E6774006844610074612000756E69007C
:104DA00074733A00206E6F0020696E0064696300BE
:104DB000617469006F6E44006174610020756E005B
:104DC000697420006C656E006774680020286200BA
:104DD00069747300293A200043532000454E410076
:104DE000424C450044435300204449005341420093
:104DF0004C45440052335700202873007064200053
:104E000063736C00206869007A293D00282029001E
:104E10000D0A4400697363006F6E6E006563740071
:104E200020616E0079206400657669006365730017
:104E30000D0A43006F6E6E006563740020285600F3
:104E400070752000746F20002B35560029206100FA
:104E50006E64200028414400432074006F202B0022
:104E6000332E33005629430074726C0041555800AC
:104E70004D4F440045204C0045445000554C4C00DB
:104E800055502000485055004C4C550050204C00C7
:104E90005652450047414400432061006E642000A3
:104EA00073757000706C790035565600505533009C
:104EB0002E33560041444300427573002068690058
:104EC000676842007573200048692D005A20300041
:104ED00042757300204869002D5A2000314D4F0063
:104EE00044452000616E6400205652004547200072
:104EF0004C45440073207300686F75006C6420009B
:104F0000626520006F6E2100466F75006E642000A0
:104F100020657200726F7200732E4D004F5349006E
:104F2000434C4B004D4953004F435300204F4B001F
:104F300020464100494C53006574200073706500A1
:104F400065643A000D0A2000312E200033304B00FA
:104F5000487A0D000A2032002E20310032354B00F5
:104F6000487A0D000A2033002E20320035304B00E5
:104F7000487A0D000A2034002E2031004D487A0076
:104F8000436C6F00636B2000706F6C00617269008E
:104F900074793A000D0A2000312E200049646C001B
:104FA00065206C006F7720002A64650066617500DB
:104FB0006C740D000A2032002E204900646C6500DC
:104FC0002068690067684F00757470007574200070
:104FD000636C6F00636B200065646700653A0D00C9
:104FE0000A2031002E204900646C650020746F0097
:104FF0002061630074697600650D0A0020322E007E
:105000002041630074697600652074006F20690098
:10501000646C6500202A640065666100756C74002C
:10502000496E70007574200073616D00706C6500CE
:1050300020706800617365003A0D0A0020312E006F
:10504000204D690064646C0065202A006465660078
:1050500061756C00740D0A0020322E0020456E0030
:1050600064535000492028007370640020636B0073
:10507000702073006B652000736D700020637300F7
:105080006C206800697A29003D28200020302E001D
:105090004D616300726F20006D656E00750D0A0032
:1050A00020312E00536E69006666200043532000B5
:1050B0006C6F77000D0A2000322E53006E69660077
:1050C000662061006C6C2000747261006666690085
:1050D000632D7000202D6600202A4200797465003F
:1050E00073206400726F7000706564002A4641008E
:1050F000494C4500442C20004E4F200044415400B0
:105100004144610074612000626974007320610091
:105110006E64200070617200697479003A0D0A00B3
:1051200020312E0020382C00204E4F004E4520000C
:105130002A646500666175006C7420000D0A200009
:10514000322E2000382C2000455645004E200D0000
:105150000A2033002E2038002C204F004444200029
:105160000D0A2000342E2000392C20004E4F4E0016
:10517000455374006F70200062697400733A0D002B
:105180000A2031002E203100202A6400656661006B
:10519000756C74000D0A2000322E2000325265001A
:1051A0006365690076652000706F6C00617269004C
:1051B00074793A000D0A2000312E200049646C00F9
:1051C00065203100202A640065666100756C7400FA
:1051D0000D0A2000322E200049646C00652030004A
:1051E0005541520054202800737064002062720000
:1051F0006720640062702000736220007278700083
:10520000206869007A293D0028202000302E4D00BA
:10521000616372006F206D00656E75000D0A2000DD
:10522000312E540072616E007370610072656E0001
:10523000742062007269640067650D000A20320004
:105240002E4C6900766520006D6F6E0069746F00EA
:10525000720D0A0020332E004272690064676500F7
:105260002077690074682000666C6F007720630007
:105270006F6E7400726F6C000A0D2000342E4100B6
:1052800075746F00204261007564200044657400ED
:1052900065637400696F6E005541520054206200CE
:1052A000726964006765520065736500742074005C
:1052B0006F206500786974005261770020554100C5
:1052C00052542000696E70007574550041525400AC
:1052D000204C49005645200044495300504C4100A1
:1052E000592C20007D2054004F205300544F500073
:1052F0004C49560045204400495350004C41590048
:10530000205354004F5050004544570041524E0026
:10531000494E47003A207000696E7300206E6F009E
:1053200074206F0070656E002064720061696E0009
:1053300020284800695A2900205245005649440057
:105340003A0D0A00496E7600616C690064206300C2
:10535000686F690063652C00207472007920610019
:10536000676169006E6D7300525320004C4F570007
:105370002C2043004F4D4D00414E4400204D4F0026
:105380004445520053204800494748002C2044001F
:1053900041544100204D4F00444541006464720077
:1053A00065737300206F6600205043004638350057
:1053B00037343F005468690073206D006F646500E6
:1053C00020726500717569007265730020616E005E
:1053D000206164006170740065724C0043442000D9
:1053E00074797000653A0D000A2031002E204800C3
:1053F00044343400373830002028750073696E005B
:1054000067205000434638003537340020494F00AC
:105410002065780070616E0064657200294C43005D
:1054200044202800747970002061640064722900AF
:10543000203D200028202000302E4D0061637200A6
:105440006F206D00656E75000D0A2000312E4C0036
:10545000434420005265730065740D000A20320039
:105460002E496E00697420004C4344000D0A200050
:10547000332E43006C65610072204C0043440D00E4
:105480000A2034002E43750072736F007220700082
:105490006F73690074696F006E206500783A2800A8
:1054A00034292000300D0A0020362E005772690082
:1054B000746520007465730074206E00756D620061
:1054C00065727300206578003A283600292038007C
:1054D000300D0A0020372E005772690074652000D5
:1054E0007465730074206300686172006163740006
:1054F00065727300206578003A283700292038004B
:105500003044690073706C00617920006C696E0032
:1055100065733A000D0A2000312E200031200D0065
:105520000A2032002E204D00756C740069706C00EA
:1055300065494E00495443004C45410052435500D3
:1055400052534F005220530045544E006F204100EB
:10555000434B2C002063680065636B00206164008E
:1055600061707400657243004C4B09004D4F53004D
:105570004909430053094D0049534F0050696E00DB
:1055800073746100746573003A474E004409330038
:105590002E33560009352E00305609004144430091
:1055A000095650005509410055580900500950004E
:1055B0000950090049094900092D09004F574400C5
:1055C000092D09002D2D090054784400092D0900EA
:1055D0005278440053434C000953440041092D00C4
:1055E000092D50004743090050474400092D090088
:1055F0002D312E0028425200290932002E28520057
:1056000044290900332E28004F52290009342E0066
:1056100028595700290935002E2847004E2909002E
:10562000362E2800424C290009372E0028505500FC
:10563000290938002E28470052290900392E280050
:105640005754290009302E0028426C006B2947006E
:105650004E440900474E44000941440043093500C7
:105660002E30560009332E0033560900565055008F
:105670000941550058096500786563007574650037
:10568000203A200020617500746F7200616E67001F
:1056900065202B004D487A00292B6B00487A2900A1
:1056A00052617700207661006C75650020666F009E
:1056B0007220420052472000284D490044493D00D5
:1056C0003132370029574100524E49004E473A00C7
:1056D00020506F0073736900626C65002062750072
:1056E00066666500726F7600657266006C6F7700A3
:1056F000416E7900206B6500792074006F20650091
:10570000786974005370610063652000746F200035
:10571000636F6E0074696E0075654E00756D620092
:10572000657220006F662000626974007320720049
:10573000656164002F777200697465003A20430048
:10574000533A0D000A2031002E204300530D0A0069
:1057500020322E00202F430053202A00646566006B
:1057600061756C0074506F0073697400696F6E002E
:1057700020696E00206465006772650065735300E0
:10578000657276006F20610063746900766557006A
:1057900061697400696E6700206163007469760056
:1057A000697479002E2E2E002A2A2000456172008D
:1057B0006C7920004578690074212A002A42610032
:1057C00075643E0031366D003A204200502043009F
:1057D000616E6E006F7420006D65610073757200FC
:1057E00065203E002031360030303000303030004F
:1057F0002C2044006F6E65002E0A0D0043616C0082
:1058000063756C0061746500643A2000090A0D003C
:1058100045737400696D6100746564003A2020006E
:10582000092062007073200047656E006572610098
:105830006C0909000909090050726F00746F630058
:105840006F6C2000696E740065726100637469009A
:105850006F6E20002D2D2D002D2D2D002D2D2D00B6
:105860002D2D2D002D2D2D002D2D2D002D2D2D001C
:105870002D2D2D002D2D2D002D2D2D002D2D2D000C
:105880002D2D2D002D2D2D002D2D2D002D2D2D00FC
:105890002D2D2D002D2D2D002D2D2D002D2D2D00EC
:1058A0002D2D2D002D2D2D002D2D2D002D2D2D00DC
:1058B0002D2D2D002D2D2D00203F0900546869004D
:1058C00073206800656C7000090909002830290000
:1058D000094C6900737420006375720072656E0074
:1058E00074206D00616372006F7320003D582F00BB
:1058F0007C580900436F6E00766572007473200057
:10590000582F720065766500727365002058090093
:105910000928780029094D00616372006F20780022
:10592000207E090053656C0066746500737409007D
:1059300009095B0009537400617274002023090097
:105940005265730065742000746865002042500041
:1059500020202000090909005D095300746F7000C0
:10596000202409004A756D00702074006F206200C9
:105970006F6F74006C6F61006465720009097B00D1
:105980000953740061727400207769007468200004
:1059900072656100642026002F25090044656C00B3
:1059A0006179200031207500732F6D0073090900A3
:1059B000097D090053746F00702061002F412F0092
:1059C0004009410055585000494E2000286C6F0096
:1059D000772F4800492F520045414400290909000A
:1059E000226162006322090053656E006420730027
:1059F000747269006E6720006209530065742000AC
:105A00006261750064726100746509000909310002
:105A100032332000632F43000941550058206100B4
:105A200073736900676E6D00656E740020286100F5
:105A300075782F004353290009093000783132006E
:105A4000332064002F4409004D65610073757200B6
:105A50006520410044432000286F6E0063652F00DD
:105A6000434F4E00542E290009306200313130007E
:105A7000095365006E64200076616C007565200036
:105A800066094D00656173007572650020667200DD
:105A900065717500656E630079090900720952002D
:105AA0006561640020672F0053094700656E65003B
:105AB0007261740065205000574D2F0053657200CD
:105AC000766F0900092F0900434C4B0020686900DC
:105AD00020680900436F6D006D616E0064686900A5
:105AE00073746F007279090009095C0009434C0066
:105AF0004B206C006F2069000956650072736900C5
:105B00006F6E69006E666F002F73740061747500AC
:105B100073696E00666F0900095E0900434C4B0013
:105B200020746900636B20006C2F4C0009426900EF
:105B3000746F72006465720020286D0073622F001C
:105B40004C534200290909002D094400415420000A
:105B5000686920006D09430068616E006765200078
:105B60006D6F640065090900095F09004441540034
:105B7000206C6F00206F090053657400206F750062
:105B8000747075007420740079706500090909004B
:105B90002E094400415420007265610064207000A9
:105BA0002F50090050756C006C75700020726500F4
:105BB00073697300746F7200732028006F6666004B
:105BC0002F4F4E00290921000942690074207200FC
:105BD000656164002073090053637200697074008A
:105BE00020656E0067696E0065090900093A0900C1
:105BF000526570006561740020652E00672E2000DC
:105C0000723A310030207600095368006F77200027
:105C1000766F6C0074732F00737461007465730089
:105C200009093B000942690074732000746F200069
:105C300072656100642F77007269740065206500E9
:105C40002E672E002030780035353B00322077005B
:105C50002F5709005053550020286F0066662F000B
:105C60004F4E290009093C00783E2F003C783D004A
:105C7000203E2F003C303E000955730065726D00D8
:105C8000616372006F2078002F6173007369670091
:105C90006E2078002F6C690073742000616C6C00BA
:105CA000A0AE20001064A00080AF2000104078005B
:105CB0006840600005003200CAC2A900F0C2B3000B
:105CC000DC5A02000000000001003700CAC2A80030
:105CD000A100200090AB2000F4730200000000003F
:105CE00000000600A0AE20001064A10080AF2000DC
:105CF000104078006840600005003200CAC2A90068
:105D0000F0C2B300DC5A02000000000001003700BE
:105D1000CAC2A800A100200090AB2000F4730200CA
:105D2000000000000000060080AF20001040780056
:105D30006840600005003200CAC2A800F0C2B3008B
:105D4000DC5A02000000000001003700CAC2A900AE
:105D5000B100200030AC2000F4730200000000000D
:105D60000000060000C0EB00C90107000080FB0036
:105D700000000600C601070000417800A0AE200028
:105D800001C4B30010C060008000EB0001003200CD
:105D90008280FB000100780000000600881F780068
:105DA0000102200000CA20009A73020000000000D7
:105DB00080AD20001040E8002C59020000000000D7
:105DC00000C2B300DC5A02000000000088AF2000CF
:105DD0009840780061C060002C590200000000006B
:105DE00000C2B300DC5A0200000000001880FB0073
:105DF0000000D100614060002C590200000000004A
:105E000000C2B300DC5A0200000000001880FB0052
:105E10004200DE00614060002C59020000000000DA
:105E200000C2B300DC5A0200000000001880FB0032
:105E30004300DE00614060002C59020000000000B9
:105E400000C2B300DC5A020000000000A0AE200037
:105E50001080FB004400DE00614060002C5902000D
:105E60000000000000C2B300DC5A02000000000085
:105E70003100200020AE20009A73020000000000D4
:105E80004F04780000000600889FBE008A9FBE0075
:105E90008C1F7800EA19020000000000541802006C
:105EA0000000000000047800EA1902000000000071
:105EB000541802000000000080047800EA19020073
:105EC00000000000541802000000000000057800E7
:105ED000EA1902000000000054180200000000004F
:105EE00080057800EA190200000000005418020042
:105EF0000000000000067800EA190200000000001F
:105F00005418020000000000000178000800E900B9
:105F1000E30F5000020036000004EB0002003700DF
:105F200080AD20000848E9000900E900E10F5000B9
:105F3000020036000004EB000500370081AF2000AE
:105F40000940E900614060001104A100914870001F
:105F50000A00E900E10F5000020036000004EB00E7
:105F60000600370081AF20000A40E9006140600070
:105F7000004040001114A100914870000B00E9009E
:105F8000E10F5000020036000004EB00060037006D
:105F900081AF20000B40E900614060004200DD005D
:105FA0001124A100914870000C00E900E10F50009D
:105FB000020036000004EB000600370081AF20002D
:105FC0000C40E900614060004300DD001134A10095
:105FD000914870000200E900E10F500008003E0007
:105FE000A0AE2000E1406100C408DD00104178004F
:105FF0000244A100014871000800E0005B003A0083
:106000008004EB00296488007103200000BC20009C
:10601000F4730200000000008901780042002000B3
:106020001100200010002000E41A0200000000000F
:1060300081AD20008048E9005103200070BF20009E
:10604000F4730200000000008901780022002000A3
:106050001100200010002000E41A020000000000DF
:1060600088AF20000040E900614060001804A100F2
:10607000184C700031042000C0C22000F4730200EC
:10608000000000008901780022002000110020009B
:1060900020002000E41A0200000000000040E90097
:1060A00061406000004040001814A100184C7000CE
:1060B00011032000F0C62000F4730200000000006D
:1060C000890178002200200011002000100020002B
:1060D000E41A0200000000000040E9006140600096
:1060E0004200DD001824A100184C7000D1012000EE
:1060F000601C2100F4730200000000008901780098
:10610000220020001100200020002000E41A0200DC
:10611000000000000040E900614060004300DD0035
:106120001834A100184C7000F1042000E093200006
:10613000F4730200000000008901780022002000B2
:106140001100200010002000E41A020000000000EE
:10615000A2AE2000614060004400DD009240780063
:106160000144A10000C97000010037000BFF0700C7
:10617000A0AE20001064A10080AD20009080FB0044
:10618000E0812000614078007600070080AF2000A9
:106190001080FB004300DE00614060004600DD002F
:1061A000A12C2000914078000164A10080C0700003
:1061B00001007800CAE2B7004F0678004F05BE0024
:1061C0004F04BE0000000600A30007000000060008
:1061D00001002000EF0F5000E08F580057003E00F4
:1061E000006001000F003700130037001E00370069
:1061F0005600370051003700500037004F0037007D
:106200004E0037004D0037004C00370022003700A9
:106210002400370026003700280037002A00370006
:106220002C0037004103200000CC2000F473020052
:10623000000000004500370071002000705620006B
:10624000F473020000000000F1002000B0182100EB
:10625000F47302000000000011C0B3000040EB0026
:1062600094000700390037007100200070562000AC
:10627000F473020000000000F1002000B0182100BB
:10628000F47302000000000011C0B3000140780068
:10629000880007002D00370080AF20001004A10007
:1062A0000E00370080AF20001004A0000B00370064
:1062B00080AF20001014A1000800370080AF20003C
:1062C0001014A0000500370080AF20001024A100AA
:1062D0000200370080AF20001024A00082AF200011
:1062E00012407800E1406000C608DD0042C2BF00F5
:1062F0000064A1000140700042E2B7009280FB0000
:106300000101D1006141610043C2BF000004A1004E
:106310000240700043E2B700C208DE00E1C0600046
:1063200081C0400043C2BF000014A10001407000C2
:1063300043E2B70099FE0700040037004102200045
:10634000E01D2000F47302000000000000000600C1
:106350000101200040062100F4730200000000004B
:10636000000006000041780041E2A900A0AE200034
:10637000104078007040600004003200CEE2A800B7
:10638000CF02A800CEC2A80003003700CEE2A900C9
:10639000CF02A900CEC2A900A8C6BF0001CEB3009B
:1063A000014060007040B300A8E6B700C9C6BF0056
:1063B000014060007040B300C9E6B700C8C6BF0026
:1063C000014060000034A000C8E6B700CAC2A800BF
:1063D000C8C2A900C902A900C8E2A800C922A90030
:1063E0000280FB001012880042A2A80082AF2000A9
:1063F00012407800E1406000C608DD0042C2BF00E4
:106400000064A1000140700042E2B7009280FB00EE
:106410000101D1006141610043C2BF000004A1003D
:106420000240700043E2B700C208DE00E1C0600035
:1064300081C0400043C2BF000014A10001407000B1
:1064400043E2B7000000EB00201288000012880031
:1064500041E2A8000000060041E2A900F0C1B3003B
:10646000A866B700C9C6BF0001CEB30001406000F6
:10647000C9E6B700C8C6BF0001406000C8E6B70063
:10648000CEE2A900CF02A900CEC2A90000000600FA
:106490000080FB004012880085C0BF000028A300D8
:1064A000FDFF3200401280008540A9000080FB0003
:1064B00000000600889FBE008A9FBE008C9FBE0021
:1064C0008046780081457800AC812000485A02005F
:1064D00000000000E0FF0700710007000D04E0006D
:1064E00007003A0042E2A80062E2A8000600370076
:1064F000E08828006857020000000000F3FF370022
:10650000E1CF560064003E0041E2A80061E2A8002D
:10651000610037000A04E00007003A00CAC2BF0069
:106520000068A30004003200D0C5B300A05A0200E6
:10653000000000001AC0B30040C2BF000058A30012
:1065400028003A0060C2BF0001C2B30001446000ED
:1065500024003A004012800080447800E14F55004A
:1065600004003A00B0C5B300A05A020000000000C9
:10657000084578000B04E000040032000980FB00AD
:106580008E5902000000000006003700C0C5B300AD
:10659000A05A02000000000009407800A05A020042
:1065A0000000000040138000004478000B04E0006D
:1065B0000A00320080C2B300A05A020000000000AE
:1065C0000880FB008E5902000000000090C2B3005A
:1065D000A05A02000000000002003700A05A02008A
:1065E0000000000040C2BF000068A30007003A009E
:1065F00060C2BF000068A30004003A000040200011
:106600001C0060000D003200050037000040200033
:106610001C00600002003A007A5A020000000000EC
:106620000000EB0000128800001388000B04E0005B
:10663000AFFF3A00C222A9000D003700565A0200EF
:1066400000000000425A020000000000E14F50002C
:10665000B0FF3A00C85A0200000000000B04E0003E
:1066600003003200F0892800685702000000000093
:106670005A00070080AD20009080FB00E0812000E0
:106680006140780037FF07004F06BE004F05BE008F
:106690004F04BE00000006001AC0B300A6FF37007A
:1066A000C8C2A800C902A800C8E2A800C922A80060
:1066B000AAC6BF0001CEB300014060006040B30035
:1066C000AAE6B700AEC6BF00014060006040B3005C
:1066D000AEE6B700A8C6BF00014060009040B3001E
:1066E000A8E6B700A9C6BF00014060000034A000C2
:1066F000A9E6B700ACC6BF00014060007040B3001F
:10670000ACE6B700ADC6BF00014060000034A00099
:10671000ADE6B70080AD20009080FB00E081200056
:10672000614278000482FB001412880081AF2000CF
:1067300011407800E1416000C619DD0042C2BF008F
:10674000F6CBB300064060000340700042E2B700A1
:106750001181FB000201D1006141610043C2BF0011
:10676000E5CFB300054060000240700043E2B7008F
:106770008000EB00211288000112880014138800A9
:1067800062C2BF00064060000340700062E2B700D2
:1067900063C2BF00054060000240700063E2B700C2
:1067A00021138800011388004112880041138800DA
:1067B0004322A9006322A9004362A80042A2A900C3
:1067C0006362A80062A2A90040C2A90060C2A90039
:1067D0004402A8006402A8000000060041E2A900EB
:1067E0004362A90061E2A9006362A900F0C1B3009D
:1067F000AA66B700AE66B700A866B700A966B7007C
:10680000AC66B700AD66B70000000600008A28003D
:10681000505702000000000000000600889FBE00E4
:106820008A9FBE008C9FBE0011C0B30080AD2000C7
:106830000148780080AF20001004A1001014A000CF
:106840001024A100A0AE20001044A000208220004F
:1068500010409000C3FE0700ECFF07006CAF200063
:10686000C85A02000000000080417800004E780005
:106870000080FB00C400DE0050AF2000014878001B
:10688000E4CF50001D01320005003E000104E0008D
:1068900008003200E1CF50004A013A0002013700FF
:1068A000E6CF50001C013200E8CF500045013A000D
:1068B00025013700E5CF51000A003E00E4CF51002A
:1068C0002E003100E1CF5100120032000C003900DF
:1068D000E2CF510011003200E3CF5100EE003A0048
:1068E00013003700EDCF510016003200EECF5100FB
:1068F0001B003200E6CF5100E7003A006C00370081
:10690000D5FE07004F06BE004F05BE004F04BE0077
:1069100000000600BDFF0700D1FF3700CCC2A90070
:1069200010C0B300DC5A020000000000CCFF3700AA
:10693000CCC2A80010C0B300DC5A02000000000066
:10694000C7FF370010C0B300DC5A0200000000008F
:106950008040EB0010C0B300D6FE0700C0FF370038
:1069600010C0B300DC5A0200000000008040EB00C1
:1069700001407800CFFE0700B9FF3700C85A020077
:10698000000000004804DD00C85A020000000000BA
:106990000080FB0000057400C85A020000000000DF
:1069A0004804DD00C85A0200000000000080FB001F
:1069B0008005740000002100800F550002003E0099
:1069C000808F5500030136000040EB00DC5A0200C6
:1069D00000000000A2FF37008004EB00ED802000E3
:1069E0001D844400C85A020000000000004C7800DA
:1069F0008904E800890F5500F9FF3A0040C0B30050
:106A00009C4F100001003A00CAC2A9000A00E00031
:106A1000070032000004EB007040800068407800FE
:106A20009BFE07000804E800880F5500FAFF3A00B3
:106A30001000200044730200000000000B00E00082
:106A4000090032008004EB00EA8020001A84440030
:106A500000C0EB008EFE0700004C78008904E800BF
:106A6000898F5500F9FF3A0040C0B3009C4F1000D9
:106A700001003A00CAC2A80010C0B300DC5A0200EC
:106A8000000000000B00E00075FF32000004EB0086
:106A90007040800068407800DC5A0200000000006E
:106AA0000804E800888F55006DFF3200F8FF3700BA
:106AB00010C0B300DC5A02000000000022C2BF0078
:106AC0000008A300FDFF320030118000004E780066
:106AD000E14F50000A003200050039008002EB004F
:106AE0006055B800E24F50000F00320066003700DA
:106AF00010C0B300DC5A02000000000058FF37004D
:106B000010C0B300DC5A0200000000000040EB009F
:106B1000DC5A02000000000010C0B300DC5A020082
:106B2000000000004EFF370022C2BF000008A30093
:106B3000FDFF3200341180004859DD00C851DE00ED
:106B4000830171004851DD000480FB00010020003A
:106B500000057100818571008502E800E38F520015
:106B6000F1FF3600044E78008002EB006044B8006C
:106B700022C2BF000008A300FDFF320034118000D4
:106B80004849DD00C841DE00830171004841DD0055
:106B90000480FB000100200000047100818471006A
:106BA0008502E800E38F5200F1FF3600044E7800C2
:106BB000F2FF2F0003002000820F5500838F5D003D
:106BC00008003E00820F5400838F5C0005003E00E9
:106BD0000A0044008B804C00820F5000838F5800C5
:106BE000040036000040EB00DC5A02000000000008
:106BF0001BFF370010C0B300DC5A02000000000089
:106C0000E00F5400E08F5C0015FF320000C2B300BB
:106C10001FFE0700C855DE000B4078001CFE070071
:106C20000A4078001AFE07000040EB0018FE07003B
:106C3000DC5A020000000000E10F5400E08F5C000D
:106C400007FF320080C2B30011FE07000B4078003E
:106C50000FFE07000A4078000DFE07000040EB0021
:106C60000BFE0700DC5A0200000000006204540022
:106C7000E0845C000A05E800E00F5400E08F5C004F
:106C8000F7FE3200E1FF37000040EB00DC5A020063
:106C900000000000F2FE37000040EB00DC5A02006A
:106CA00000000000EEFE37006FC06100004EE800FB
:106CB00010C0B300DC5A02000000000040AF20000A
:106CC0000048EB001C04E000E5FE32000004780000
:106CD00069AF2000C85A020000000000ECFD070068
:106CE000DC5A0200000000001840E800004C780068
:106CF000994F5000DAFE3100F6FF3700034078006C
:106D0000A07702000000000010C0B300DC5A0200AF
:106D100000000000D2FE370067C06100004E78001E
:106D200081AD2000804878000080FB002182200097
:106D300060C078008BFD070010C0B300DC5A020071
:106D400000000000C6FE370081AF20001104A10042
:106D50001114A1001124A100A0AE20001044A10034
:106D60000381FB000228A300010032001104A000EF
:106D70000218A3000200320080AF20001014A0000F
:106D80000308A3000200320080AF20001024A000FE
:106D90000238A30002003A00A0AE20001044A00078
:106DA00080AD20009080FB002082200061407800B0
:106DB0006CFD070010C0B300DC5A020000000000A8
:106DC000A7FE37000040EB00DC5A02000000000084
:106DD000A3FE37000A00E00008FF3200FEFE370085
:106DE000881F7800B0760200000000000004E00078
:106DF0001A00320032C2BF000038A3000400320083
:106E00003100200040CF20009A73020000000000F3
:106E100032C2BF000028A30004003200310020006D
:106E200070CF20009A73020000000000A6760200D6
:106E3000000000000004780032C2BF000018A30068
:106E40000B003200F1002000A0CF20009A73020056
:106E5000000000003222A90005003700F1002000E8
:106E600090D020009A730200000000000004EB00A4
:106E7000080078004F047800000006009A760200AF
:106E8000000000000000EB0000000600881F7800F2
:106E900001022000F0DB20009A73020000000000D5
:106EA00088AD2000184078002C5902000000000036
:106EB00000C2B300DC5A0200000000001840780055
:106EC000E94F500007003A00C0118000E25802006C
:106ED0000000000000C2B300DC5A02000000000005
:106EE000090037000080FB0000004000E1AA2000FC
:106EF00060807800E25802000000000000C2B30089
:106F0000DC5A02000000000028D3200098407800DE
:106F100063C060002C5902000000000000C2B300F2
:106F2000DC5A0200000000001880FB004200DE0076
:106F3000614060002C5902000000000000C2B30054
:106F4000DC5A0200000000001880FB004300DE0055
:106F5000614060002C5902000000000000C2B30034
:106F6000DC5A020000000000A0AE20001080FB00F0
:106F70004400DE00614060002C5902000000000067
:106F800000C2B300DC5A0200000000003100200003
:106F900020AE20009A730200000000004F04780029
:106FA00000000600889FBE008A9FBE008C1F7800EC
:106FB000EA1902000000000054180200000000005E
:106FC000000478000006EB00EA0F500005003A00CC
:106FD000EA1902000000000054180200000000003E
:106FE00000067800EA1902000000000054180200B0
:106FF0000000000080047800EA1902000000000090
:10700000541802000000000000057800EA19020090
:107010000000000054180200000000008005780005
:10702000EA190200000000005418020000000000ED
:10703000800178000800E900E90F500002003600E6
:107040000004EB000200370080AD20000848E90092
:107050000900E900E30F5000020036000004EB00D5
:107060000600370020D320008940E900E3C060001B
:10707000C2CFB3001048610010C870000A00E900D8
:10708000E10F5000020036000004EB00060037005C
:1070900021D320000A40E900614060004200DD0089
:1070A0001124A100914870000B00E900E10F50008D
:1070B000020036000004EB000600370021D3200058
:1070C0000B40E900614060004300DD001134A10085
:1070D000914870000300E900E10F500008003E00F5
:1070E000A0AE2000E1C06100C408DD0010417800BE
:1070F0000244A100014871000800E0005B003A0072
:107100000004EB0028648800D1082000608720007C
:10711000F47302000000000088017800A200200043
:107120001100200010002000E41A020000000000FE
:107130000040E90081AD200080487800E94F500010
:107140000B003A00C1012000F0142100F47302008A
:107150000000000088017800F2FF270011002000E5
:1071600020022000E41A020000000000000678005F
:107170004105200080D120009A7302000000000029
:107180008001EB00420020001100200010002000D0
:10719000E41A02000000000028D320000040E900AB
:1071A00063406000C1CFB30018CC6000184C700081
:1071B00011022000C0D620009A73020000000000D7
:1071C0008001EB00220020001100200010002000B0
:1071D000E41A0200000000000040E9006140600085
:1071E0004200DD001824A100184C7000210320008B
:1071F000D0D820009A730200000000008001EB004C
:10720000220020001100200010002000E41A0200DB
:10721000000000000040E900614060004300DD0024
:107220001834A100184C7000F1042000E0932000F5
:10723000F4730200000000008001EB002200200037
:107240001100200010002000E41A020000000000DD
:10725000A2AE2000614060004400DD009240780052
:107260000144A10000C970000100370007FF0700BA
:1072700080AD200090417800E9CF510010003A0025
:1072800023D320001381FB004212DE004311DE00F5
:1072900061416100A0AE20009080FB00C408DE00C8
:1072A000E1C060006142620093417800E3C1610087
:1072B0000C0078001E76020000000000120037006B
:1072C00025D320001581FB004212DE004311DE00B1
:1072D00061416100A0AE20009080FB00C408DE0088
:1072E000E1C060000380FB0000004000E3AA200032
:1072F000608079006142620095427800E3C16200DB
:107300001E7602000000000020D32000104078000C
:1073100063406000E34F500003003A0091C0B300A7
:1073200090AD2000014878007E7602000000000049
:10733000C111800040118000808F50000400310096
:1073400001022000B0162100F473020000000000CA
:107350004F0678004F05BE004F04BE000000060037
:10736000867602000000000000000600889FBE0034
:1073700000047800E20F50005700320005003E0084
:107380000000E00008003200E10F500079003A00F0
:107390000E003700E30F500008003200E40F5000E9
:1073A00074003A0064003700A1062000F0DD2000E0
:1073B0009A7302000000000072003700C062A9004A
:1073C000C082A800C8C2A800C902A900B10020005C
:1073D00090E42000F473020000000000D1002000BF
:1073E00040E52000F4730200000000008A740200EF
:1073F000000000000000E000620032003222A9001C
:10740000D9FF2F0032C2BF000008A30005003200E0
:1074100023C2BF000018A30002003A00B011800090
:1074200020118800425A020000000000E14F500085
:1074300007003A0033C2BF000018A30004003A005E
:10744000C85A0200000000000080FB00A011880064
:1074500032C2BF000018A30003003A0022C2BF00DE
:107460000018A300070032008004FD003222B6009D
:107470008004FD008004FD002222B6008004FD008F
:10748000C222A900E30F5400DEFF3A00212C2000A5
:1074900091407800C408DE00E1806000CBC2BF00EC
:1074A0000004A10001407000CBE2B700CAC2BF00D7
:1074B0004600DE00610060004300DD00212C20005A
:1074C000914078000134A10080C070000100780074
:1074D000C2E2B700CBFF3700E100200010E6200039
:1074E000F473020000000000F1002000B018210039
:1074F000F4730200000000003222A90032C2BF0073
:107500000008A3000500320023C2BF000018A3003A
:1075100002003A00B011800020118800425A020097
:1075200000000000E14F5000F4FF3A00C85A02008A
:107530000000000013003700867602000000000003
:107540000000EB00920007007E76020000000000C1
:10755000C111800040118000808F5000090031006F
:1075600001022000B0162100F473020000000000A8
:107570000400370041022000E01D2000F4730200E7
:10758000000000004F04BE00000006003222A900E7
:1075900020D320001044A000A0AE20001024A000A2
:1075A000C1012000F0E62000F4730200000000009A
:1075B0000000060020D320001044A100A0AE20004F
:1075C0001024A10041012000B0E82000F473020063
:1075D0000000000000000600881F78000004EB0097
:1075E0002C00370020D3200010407800704060004D
:1075F0002500320080822800685702000000000049
:1076000061002000806620009A73020000000000E4
:1076100032C2BF000038A300040032003100200055
:1076200040CF20009A7302000000000032C2BF0069
:107630000028A300040032003100200070CF200099
:107640009A73020000000000A6760200000000000D
:10765000947202000000000032C2BF000018A300B4
:1076600005003200F1002000A0CF20009A73020034
:10767000000000003222A900808228006857020022
:107680000000000002003700A676020000000000A3
:1076900018002000B0760200000000000004E000A6
:1076A000D0FF3A00080078004F0478000000060080
:1076B000B1002000B00A2100F473020000000000B5
:1076C000000006000000EB00F00888008008880039
:1076D0008100200081088800400888003008880068
:1076E000B0088800A0088800F108880000000600A3
:1076F00011E1A9001FE1A900F0C1B3008666B7003F
:107700000000EB00F008880080088800300888003E
:1077100040088800000006000002BE0011002000A2
:10772000E08228001001BE00840F5100858F5900AF
:1077300010003600C208DD00A082280080804000D2
:1077400061BB9700F1BB970006005100878059008C
:107750008100D1000080D3000600400087804800EF
:10776000800F5200818F5A0007003E000601BE00C4
:10777000050037008100E80064004000EF8F5000F2
:10778000E8FF3A006011B8000200BE0000000600E9
:10779000889FBE008A9FBE008C9FBE008006780036
:1077A000CAE2A900C8E2A8000000E00004003A0014
:1077B0003101200020202100F473020000000000AD
:1077C000CA42E20007003D006300370000000000ED
:1077D000CA42E20003003D0022C2BF000008A3002D
:1077E000FAFF320022C2BF000008A30008003200E6
:1077F00030118000BEFF0700E10020005021210071
:10780000F4730200000000006044B8005600370026
:107810008004EB006055B80008C8B3000006EB0018
:10782000A8FF0700CAC2BF0008406000FDFF320089
:107830001FE1A80011E1A80001C8B300CAC2BF003F
:1078400001406000FDFF3A0011E1A9001FE1A9001D
:10785000F0C1B3008666B700FC0888008C08880079
:107860004008800001002000C000DD000000200072
:107870003208800002004000E08048000900E0007B
:1078800007003200E00F5500E08F5D00030032007A
:107890008A0F50008B8F5800010031000005BE0098
:1078A0008904E800F98F5400DDFF3A0090FF0700DB
:1078B0000A01BE0000402200410F20002406020001
:1078C000000000000004BE000D00E00026003A00A9
:1078D000009F240021002000800F5400818F5C0055
:1078E00005003600F102200030222100F47302006E
:1078F000000000001C003700F100200020252100BE
:107900009A730200000000000800BE00B257020097
:10791000000000004100200000272100F473020055
:1079200000000000F1002000102621009A730200E0
:10793000000000000800BE0077FF0700B2570200F9
:10794000000000004100200000272100F473020025
:10795000000000000400370022C2BF000008A3009E
:107960009AFF32009FFF37000800BE004F06BE009E
:107970004F05BE004F04BE0000000600A086280090
:10798000505702000000000000000600889FBE0063
:107990008A9FBE008C1F780021D32000C0CFB30087
:1079A000914860001124A1001134A100A0AE200074
:1079B0001044A00010568000606988001144A100A6
:1079C0001181FB004212DE004311DE0061416100C3
:1079D0006142620091407800E3C1600011C0B300D1
:1079E0001E760200000000007E760200000000000B
:1079F000E2FF070028D320000AD32000ABAE20000E
:107A0000B0760200000000000004E0000A0032002E
:107A10009840780070C0600005003200A676020031
:107A200000000000DC5A02000000000002003700E5
:107A3000A67602000000000032C2BF000018A300BA
:107A4000010032003222A900425A02000000000068
:107A5000E14F5000EAFF3A00C85A0200000000005F
:107A600080417800004D78000080FB00C400DE00FB
:107A7000F0D2200001487800E4CF50008A003200A4
:107A800005003E000104E0000A003200E1CF500092
:107A9000E1003A006C003700E6CF50008900320068
:107AA000DD00390068C05000E14F5000DA003E00B0
:107AB000A5003700E2CF51001500320005003E005E
:107AC0000304E0000A003200E1CF51005A003A00FE
:107AD0000D003700E7CF51001B003200EFCF5100FF
:107AE0003D003200E3CF510053003A00110037004F
:107AF00086760200000000004F0678004F05BE00A9
:107B00004F04BE00000006009CFF0700BCFF3700CA
:107B100010C0B300DC5A02000000000032C2BF00F7
:107B20000018A300010032003222A9001844A0006E
:107B3000B3FF37001844A10010C0B300DC5A0200A4
:107B400000000000AEFF370010C0B300DC5A020096
:107B5000000000008676020000000000C85A020003
:107B6000000000004800DD006069880010C0B3001C
:107B7000DC5A020000000000C85A020000000000A9
:107B80000080FB006169800001007000606988006E
:107B90001881FB004212DE004311DE0061416100EA
:107BA0009B80FB00C408DE00E1C06000614262000F
:107BB00098427800E3C162001E76020000000000D7
:107BC0007E7602000000000010C0B300DC5A020004
:107BD000000000008AFF370010C0B300DC5A02002A
:107BE000000000003222A90032C2BF000008A3003A
:107BF0000500320023C2BF000018A30002003A00B3
:107C0000B011800020118800425A020000000000DC
:107C1000E14F5000F4FF3A0033C2BF000018A30048
:107C2000F1FF3A00C85A0200000000000080FB008B
:107C3000A0118800ECFF37000040EB00DC5A020086
:107C4000000000006EFF37006FC06100004DE800CB
:107C500010C0B300DC5A020000000000E0D2200097
:107C60000048EB001A04E00065FF32008004780051
:107C70000CD32000C85A0200000000000080FB0066
:107C80009A7602000000000010C0B300DC5A020027
:107C9000000000001940E800804C78009C4F500024
:107CA00057FF3100F3FF370003407800A077020050
:107CB0000000000010C0B300DC5A02000000000009
:107CC0004FFF37006FC0610001D32000804878006B
:107CD000EA4F500002003600A0C0B3008048780090
:107CE0001A80FB000000400021AC2000608078007A
:107CF0006069880086760200000000001881FB00A1
:107D00004212DE004311DE00614161009B80FB00F6
:107D1000C408DE00E1C0600060698000614262006A
:107D200098427800E3C162001E7602000000000065
:107D30007E7602000000000010C0B300DC5A020092
:107D4000000000002EFF370021D32000C4CFB30075
:107D5000914862001124A1001134A1001B44A1002C
:107D60000381FB000238A300050032009142780035
:107D700063C062000014A00084C8620091487000D3
:107D80000228A300060032009840780063C060001B
:107D90000004A000C1CFB30018CC6000184C7000E4
:107DA0000218A300010032001824A0000308A30059
:107DB000010032001834A0000248A30001003A007C
:107DC0001B44A00086760200000000001881FB0022
:107DD0004212DE004311DE00614161009B80FB0026
:107DE000C408DE00E1C0600060698000614262009A
:107DF00098427800E3C162001E7602000000000095
:107E00007E7602000000000010C0B300DC5A0200C1
:107E100000000000FAFE37000040EB00DC5A0200D0
:107E200000000000F6FE3700E08D280050570200E9
:107E30000000000000000600889FBE008A9FBE0070
:107E40008C1F7800A1AE2000114078000034A10002
:107E50000044A0008048780018C0B30080AD200026
:107E60000848780081C0B30090AD20000148780038
:107E700020C0B300C1D420008048780080C0EB004F
:107E8000AA5E020000000000C922A900C902A900E0
:107E9000C8E2A80008407800D66002000000000098
:107EA000E1FF07000AD52000ECD42000C85A0200E8
:107EB0000000000080417800004D78000080FB0049
:107EC0004400DE00F1D4200080487800E34F5000E9
:107ED000C700320004003E00E14F5000860032002F
:107EE000BA003E000B003700E64F5000720232002D
:107EF00003003E00E44F5000A3023A00670237003F
:107F0000E84F50007B023200EA4F50009E023A00D8
:107F1000D80037000380FB0001002000ED0F500067
:107F2000E08F580070003E00006001009A023700A8
:107F30000C0037000D003700120037001700370023
:107F40001D003700230037003A0037003E0037009D
:107F500042003700480037004E0037005400370019
:107F60005A003700B0FF0700D0FF37001C5F020047
:107F70000000000010C0B300DC5A02000000000046
:107F8000CAFF3700505F02000000000010C0B300BD
:107F9000DC5A020000000000C4FF37000040EB0084
:107FA000D66002000000000010C0B300DC5A0200DE
:107FB00000000000BDFF370010C0B300D660020013
:107FC0000000000010C0B300DC5A020000000000F6
:107FD000B6FF3700C0D4200021C0B30090CF1000FE
:107FE00004003A001460020000000000004E780017
:107FF00004003700F00F20006C5F0200000000005A
:10800000004E7800A0AE200010407800684060006C
:10801000040032001C80FB007273020000000000AC
:10802000004E78001C407800DC5A0200000000007E
:108030009EFF37005660020000000000DC5A02007C
:108040000000000099FF3700E2600200000000001D
:10805000DC5A02000000000094FF370010C0B3009B
:10806000986002000000000010C0B300DC5A02005B
:10807000000000008DFF37000040EB00CA600200E6
:108080000000000010C0B300DC5A02000000000035
:1080900086FF370010C0B300CA6002000000000075
:1080A00010C0B300DC5A0200000000007FFF370060
:1080B0000040EB00BE6002000000000010C0B300F2
:1080C000DC5A02000000000078FF370010C0B30047
:1080D000BE6002000000000010C0B300DC5A0200C5
:1080E0000000000071FF37000040EB00DC5A020086
:1080F000000000006DFF37006FC06100004DE80018
:1081000010C0B300DC5A020000000000004EEB007B
:108110001A04E00065FF3200D9D42000ABAE200085
:10812000C85A02000000000080407800804C7800AF
:108130001B41780068406100040032000180FB00B0
:108140007273020000000000804C7800C0D4200050
:1081500021C0B30090CF100007003A001980FB0047
:10816000CC5F02000000000010C0B300DC5A020027
:108170000000000010003700D8D420001880FB0059
:108180006C5F02000000000080407800004C780026
:108190001B41780068406100040032000180FB0050
:1081A0007273020000000000004C78001940780053
:1081B000DC5A0200000000001C40E800004E78007D
:1081C0009A4F500039FF3100D5FF37006FC0610072
:1081D0000040E800004D78009860020000000000B8
:1081E00010C0B300DC5A0200000000002FFF37006F
:1081F0006FC06100004DE80010C0B300DC5A0200FF
:1082000000000000C85A020000000000F1D4200065
:1082100080487800004EEB001A04E00011003200A4
:1082200001047800E9D420001804E00004003D00B7
:1082300010C0B3007A6002000000000003003700A5
:108240000040EB007A600200000000001840780057
:10825000004C40001940E800804C78009A4F5000D4
:10826000F1FF390010C0B300DC5A0200000000002A
:108270000EFF370040CAB30080CF51001400320017
:1082800004003E006440500080CF51007F013A005E
:108290000700370050CAB30080CF51009800320069
:1082A00000C0E80080CF510078013A00ED003700AF
:1082B000C85A02000000000061AD2000804878002C
:1082C00010C0B300DC5A020000000000F7FE3700C7
:1082D00060AD200010407800E14F500003003200F4
:1082E000E24F500082003A002A003700C85A0200CC
:1082F000000000000080FB006300B900506A8800A5
:108300000001EB00226A88000000E0000C0032004F
:1083100082007800E980200019844000C85A0200D9
:1083200000000000004C7800206A80008000E80017
:10833000216A8800506A8000808F5000F6FF390063
:108340008000EB00216A8800506A80000000E00095
:108350000C0032007040800001004000204190007D
:108360009040900010407800D7010700206A8000FC
:10837000E3004000216A8800506A8000808F50002E
:10838000F4FF390010C0B300DC5A02000000000006
:10839000C6FE3700C85A0200000000000080FB0043
:1083A0004200DD00506A88008000EB00216A8800EE
:1083B0000B003200E980200019844000C85A0200F6
:1083C00000000000004C7800206A80008000E80077
:1083D000216A8800506A8000808F5000F6FF3900C3
:1083E0000000EB00206A8800506A80000000E00076
:1083F0003B0032000040EB007A6002000000000009
:108400000040EB007A600200000000000040EB003A
:108410007A600200000000000040EB007A60020079
:1084200000000000216A80007040800061407800F8
:108430000080FB00CC5F0200000000007040800064
:10844000216A800001004000104090000080FB0085
:10845000CC5F02000000000070408000216A8000B4
:1084600001004000204090000080FB00CC5F020033
:1084700000000000226A8000E0802000100041001F
:1084800063004000904078006FC86000004EEB0031
:108490007040800000004100304090000004E00087
:1084A0000A003200E8D42000B80107001840E800B4
:1084B000004C7800226A8000714080008280400079
:1084C000B1409000814F5000F7FF3900E4004100B7
:1084D000216A8800506A8000808F5000C5FF3900F3
:1084E00010C0B300DC5A0200000000006FFE37002D
:1084F0000040EB00DC5A0200000000006BFE370079
:1085000060AD200010407800E14F500003003200C1
:10851000E24F500065FE3A0030003700C85A0200B2
:10852000000000000080FB00506A8800C85A02006A
:1085300000000000F1D42000804878000000EB002B
:10854000206A8800506A80000000E00057FE320078
:10855000D8D42000E9D42000F0D42000104C7800BA
:10856000804CEB001880FB000008A30004003200E0
:1085700010C0B3007A600200000000000300370062
:108580000040EB007A600200000000001880FB0051
:108590000000D100004C78001940E800804C7800C1
:1085A000E34F5000EFFF36001460020000000000AF
:1085B0001460020000000000DC5A0200000000000D
:1085C000206A80000000E800206A8800516A80006C
:1085D000810F500035FE3100DFFF3700C85A02001E
:1085E000000000008080FB00516A88008000EB00E2
:1085F000216A88000004E0002CFE320022C0B30093
:1086000060B92000A10B20009F010700CB010700EB
:1086100022C0B30060BB2D00A10B20009A0107000F
:1086200022C0B300603D2D00A10B20009601070081
:10863000C201070022C0B30060BB2000A10B2000D4
:1086400091010700BD010700206A80000000E800DA
:10865000206A8800516A8000810F500013FE3100AB
:10866000E6FF3700C85A0200000000000080FB004F
:10867000406A8800C85A0200000000000081FB0028
:10868000326A880060AD200010407800E24F500050
:1086900005003A00406A80006500B9000000410012
:1086A000506A880014003700E14F500006003A007D
:1086B000406A8000000040000000410000004000CF
:1086C000506A88000C003700E34F500006003A0063
:1086D000406A8000000040000000410000004000AF
:1086E000506A8800040037000040EB00DC5A0200AA
:1086F00000000000EDFD37008000EB00216A8800DB
:10870000506A80000000E0000B003200E980200089
:1087100019844000C85A020000000000004C780094
:10872000206A80008000E800216A8800506A80008A
:10873000808F5000F6FF3900306A80000000E000B2
:108740000300320010C0B300DC5A02000000000039
:108750000000EB00206A880068AD20004000370070
:1087600070408000E2407800E1CF500021003A00E4
:1087700098407800E3CF500009003A000200400022
:1087800030419000A0409000104090009A000700F7
:10879000206A800064004000206A880030003700B2
:1087A000E1CF500009003A00020040003041900043
:1087B000A040900010409000C3000700206A800095
:1087C00064004000206A880025003700E2CF500096
:1087D00023003A0002004000C04090000000E80082
:1087E00000010700206A800065004000206A8800C0
:1087F0001B003700E2CF500019003A009840780083
:10880000E3CF500007003A00020040001040900003
:1088100065000700206A80000080E800206A880068
:108820000F003700E1CF500007003A00020040007F
:10883000104090008C000700206A80000080E80053
:10884000206A880006003700E2CF500004003A009A
:108850003A010700206A80000000E800206A8800D2
:10886000226A8000506A8000800F5100BCFF3900EE
:10887000306A80000000E0008CFD3A0010C0B300B8
:10888000DC5A02000000000088FD37000040EB00C9
:10889000DC5A02000000000084FD3700034078002D
:1088A000A07702000000000010C0B300DC5A0200F4
:1088B000000000007DFD3700E3C06100014D78003D
:1088C00080AD200001487800C0D42000104078001E
:1088D000AA5E02000000000010C0B300D6600200D3
:1088E0000000000010C0B300DC5A020000000000CD
:1088F0006EFD3700A2AE2000124078000040A100BB
:10890000004978008380FB000138A30002003A0090
:108910000044A00000497800C2D4200020C0B30069
:10892000004978000128A3000200320030C0B300E3
:1089300000497800A2AE2000124078000030A1006B
:10894000004978000118A300020032000034A000A2
:108950000049780080AD200090407800C0D420000D
:1089600010407800AA5E02000000000010C0B300B2
:10897000D66002000000000010C0B300DC5A020004
:108980000000000049FD37000040EB00DC5A020007
:108990000000000045FD37004F0678004F05BE007F
:1089A0004F04BE0000000600889FBE00004478000F
:1089B00069C0B300614064007A60020000000000FA
:1089C0000880FB000004D1008944E900F9FF3A0067
:1089D0001460020000000000DC5A020000000000E9
:1089E0001460020000000000DC5A020000000000D9
:1089F0004F04BE0000000600889FBE008A9FBE0094
:108A00008C1F780000447800814578000246780089
:108A100000C8B3000045640069C0B3006140640051
:108A20007A600200000000000880FB000004D10012
:108A30008944E900F9FF3A000A04E00006003A0020
:108A40000B80FB00CC5F0200000000000C80FB00EC
:108A5000CC5F0200000000004F0678004F05BE000A
:108A60004F04BE0000000600889FBE00004478004E
:108A700049C0B3000808A3000400320010C0B300CE
:108A80007A60020000000000030037000040EB00A5
:108A90007A600200000000000880FB000004D100A2
:108AA0008944E900F3FF3A0014600200000000006E
:108AB0001460020000000000DC5A02000000000008
:108AC0004F04BE0000000600889FBE008A9FBE00C3
:108AD0008C1F7800004478008145780002467800B9
:108AE0000080FB004605DE008044EB000F003700ED
:108AF000E3CF54000D003A000A04E0000A003200FF
:108B000010C0B300CA600200000000000A80FB0031
:108B100020730200000000000040EB00CA60020069
:108B2000000000000C00370039C0B3000808A300A3
:108B30000400320010C0B3007A60020000000000A0
:108B4000030037000040EB007A60020000000000E4
:108B50000880FB000004D1008944E800E3CF540002
:108B6000E3FF36000B80FB00CC5F0200000000003A
:108B70000C80FB00CC5F0200000000004F06780074
:108B80004F05BE004F04BE00000006000040EB0091
:108B90007A600200000000000040EB007A600200F2
:108BA000000000000040EB007A60020000000000BE
:108BB0000040EB007A600200000000000000EB00C3
:108BC000CC5F0200000000000000EB00CC5F020060
:108BD000000000000000EB00CC5F0200000000007D
:108BE00000000600889FBE000004780081447800E1
:108BF0000040EB007A600200000000000040EB0043
:108C00007A600200000000000040EB007A60020081
:108C1000000000000040EB007A600200000000004D
:108C20001880FB00CC5F020000000000184090009C
:108C30000080FB00CC5F0200000000002840900094
:108C40000080FB00CC5F0200000000006FC06400E9
:108C50000041E900E14F4100090032000244780080
:108C60000080EB000090B900004041008044E90022
:108C7000C6FF07000844E90088CF5400FCFF3A0013
:108C80004F04BE0000000600889FBE008A1F7800C7
:108C90000004BE00024578000040EB007A6002004C
:108CA000000000000040EB007A60020000000000BD
:108CB0000040EB007A600200000000000040EB0082
:108CC0007A60020000000000080078007273020061
:108CD00000000000CC5F0200000000004849DD00F9
:108CE0004840DE0000007100C848DE0072730200D8
:108CF00000000000CC5F020000000000404CDE00DD
:108D0000080078007273020000000000CC5F0200CF
:108D1000000000006F456500050032000044EB00D4
:108D20009AFF07000844E800884F5500FCFF3A000E
:108D30004F0578004F04BE0000000600881F780031
:108D400010C0B3007A600200000000000040EB0099
:108D50007A600200000000000040EB007A60020030
:108D6000000000000040EB007A60020000000000FC
:108D70000000EB00CC5F0200000000001460020065
:108D800000000000000478001460020000000000F1
:108D9000DC5A02000000000008407800DC5A0200A3
:108DA0000000000079FF070078FF07004F047800FB
:108DB00000000600005880000000E00011003200B2
:108DC00000C2B300DC5A02000000000031002000A5
:108DD000304120009A7302000000000000C2B3007E
:108DE000DC5A020000000000F05780000000E000A4
:108DF00002003A007A600200000000000000EB0070
:108E0000005888008040EB00F05780000000E00030
:108E100003003A0014600200000000008040780067
:108E200010002000005888000180FB0000000600B0
:108E3000881F780000047800005880000000E000DF
:108E40001100320000C2B300DC5A02000000000032
:108E500031002000304120009A7302000000000021
:108E600000C2B300DC5A020000000000F05780008E
:108E70000000E00002003A007A60020000000000FA
:108E80000000EB0000588800F05780000000E00070
:108E900006003A0008007800CC5F020000000000E5
:108EA00056600200000000000084FB0000C2B30016
:108EB000DC5A0200000000000800E00006003A0052
:108EC00031002000304120009A73020000000000B1
:108ED00000302000050037004100200060412000E4
:108EE0009A73020000000000001020004F04780078
:108EF00000000600005880000000E0000F00320073
:108F000041002000604120009A7302000000000030
:108F1000608A28006857020000000000F0578000B7
:108F20000000E00003003A0010C0B3007A600200C5
:108F3000000000000000EB0000588800F05780009F
:108F40000000E0000F003A001C5F0200000000007B
:108F50000000E0000B00320091002000C020200043
:108F60009A730200000000005101200050212000EF
:108F70009A73020000000000608A2800685702000F
:108F800000000000D1002000A0412000F473020086
:108F90000000000000000600005880000000E00013
:108FA0000F00320041002000604120009A7302004F
:108FB00000000000608A28006857020000000000DE
:108FC000F05780000000E00003003A0010C0B3003A
:108FD0007A600200000000000000EB0000588800EA
:108FE000F05780000000E00002003A00505F0200ED
:108FF00000000000C100200070422000F473020055
:10900000000000000000060001012000404F200089
:109010009A730200000000000040EB002C5902008F
:109020000000000000C2B300DC5A02000000000093
:1090300080AD2000104078002C5902000000000094
:1090400000C2B300DC5A020000000000708A280051
:10905000685702000000000000000600881F78002A
:109060000000EB00F0578800EA1902000000000041
:109070005418020000000000800078000000E900A1
:10908000E30F500004003E0080AD20000148E900DD
:109090000100E00010003A000004EB0028648800A2
:1090A000F8578800B103200080452000F4730200C7
:1090B000000000008801780042002000110020001C
:1090C00010002000E41A02000000000081AD200022
:1090D0008048E9000B003700818120003000230028
:1090E000910F100004003E00510320003049200081
:1090F0009A73020000000000C3FF07000000EB00AD
:1091000000588800A0AE20001044A000F057800056
:109110000000E00009003A00C922A800C902A80026
:10912000CB02A900CB22A90080AD2000904078009E
:1091300020C0B300AA5E0200000000004F047800C7
:10914000000006000000EB0000588800F057800087
:10915000E10F500001003A0007E2A90000000600FC
:10916000889FBE00E10F5000090032000300390063
:10917000E20F50006B003A005B0037005103200003
:10918000405020009A730200000000006900370080
:109190008040EB0000302000EA6002000000000088
:1091A000E102200090532000F47302000000000050
:1091B000CBC2BF000008A30005003200CBC2BF0035
:1091C000190020000004EB000018A3000C003A0076
:1091D00091002000C02020009A73020000000000CF
:1091E00051012000502120009A730200000000006D
:1091F000608A280068570200000000004D00370018
:10920000F05780000000E00008003A001C5F0200F8
:109210000000000008007800CC5F020000000000A1
:1092200056600200000000008084FB000900E0009E
:1092300020003A000800780094720200000000004C
:1092400080C2B300DC5A0200000000000880D10098
:1092500094720200000000000808A30004003A0015
:10926000908A280050570200000000000B003700D1
:10927000F05780000000E00005003A001460020092
:109280000000000010C0B3007A600200000000007F
:10929000C08A28005057020000000000708A280091
:1092A000505702000000000000C2B300DC5A020068
:1092B00000000000F05780000000E00002003A00CB
:1092C000505F0200000000000804E80000102000C9
:1092D000800F5400CAFF3A00608A280068570200D5
:1092E0000000000013003700F0578000E10F50002D
:1092F00001003A0007E2A90071002000705620002A
:10930000F473020000000000F1002000B0182100FA
:10931000F47302000000000010C0B3000C0007004E
:109320000400370041022000E01D2000F473020019
:10933000000000004F04BE0000000600B100200045
:10934000600B2100F4730200000000000000060022
:10935000E4874700889FBE008A9FBE008C9FBE00A6
:109360008E1F780090F79F00485A0200000000000E
:10937000C922A800C902A800CB02A900CB22A900DB
:1093800062A0A80062C0A8008660A900CBC2BF008E
:109390000000D100B12C20009140780061466000AF
:1093A00061C460000047EB008E4678008EF79F0096
:1093B000060037000B4678000A4478000047EB00AF
:1093C000020037000B4678000A44780086C0BF00D0
:1093D0000038A3000E003A00565A020000000000B8
:1093E000425A0200000000000004E000F7FF3200D3
:1093F000C85A02000000000062A0A90062C0A900D3
:109400009FF097000104E00057003200530037003E
:109410008660A900CBC2BF000000D100E10460005B
:1094200089457800CBC2BF006140600000457800EC
:109430000E04E0002F0032000804E0002F003A0084
:109440000004E000DFFF3200E7CF56000B003E00D3
:109450000FF097000040400080F79F000904E000F3
:10946000020032000004A00080F79F008D46E80053
:109470000B4678000A447800D4FF37001FF09700AD
:109480000004E000050032008FF097000180FB002F
:109490008E5902000000000006003700C0C5B3006E
:1094A000A05A0200000000000FF09700A05A02002E
:1094B000000000000904E00007003200D0C2B30041
:1094C000A05A0200000000000B4678000A44780011
:1094D0008046EB00BDFF3700B0C2B300A05A0200C7
:1094E000000000000B4678000A4478008046EB003C
:1094F000B6FF37000804E000AEFF32000004E000D1
:10950000B0FF32000C04E0000A0032000904E00061
:10951000ACFF3A00B0C5B300A05A02000000000042
:109520000B4678000A4478001EC0B30089467800D4
:10953000A6FF37000904E000A2FF3200D0C5B30047
:10954000A05A0200000000000B4678000A44780090
:109550000047EB008E4678009CFF3700608A2800A9
:1095600068570200000000004F0778004F06BE0059
:109570004F05BE004F04BE004F00B10000000600C2
:10958000F08A28005057020000000000000006008A
:10959000889FBE008A9FBE008C9FBE008E1F7800F1
:1095A000C922A800C902A800CB02A900CB22A900A9
:1095B000C8C2A900A1AE2000114078000034A1006B
:1095C0000044A0008048780080C0EB0020C0B300B9
:1095D000AA5E020000000000E9FF0700CAAF2000F9
:1095E000AEAE2000C85A02000000000080417800A2
:1095F000004D78000080FB004400DE00B1AF200089
:1096000080487800E14F5000D20032000500390058
:10961000E44F5000F1003200E64F5000F6003A00EF
:10962000E50037000380FB0001002000EF0F500031
:10963000E08F5800C3003E0000600100F5003700D5
:109640000E0037000F0037001400370019003700F4
:10965000BC0037001C00370022003700280037000C
:109660007D003700B7003700B6003700B50037007F
:10967000B4003700B3003700AC003700C0FF07006C
:10968000D8FF37001C5F02000000000010C0B300CC
:10969000DC5A020000000000D2FF3700505F0200D9
:1096A0000000000010C0B300DC5A020000000000FF
:1096B000CCFF37001460020000000000DC5A0200FA
:1096C00000000000C7FF37000040EB007A60020096
:1096D0000000000010C0B300DC5A020000000000CF
:1096E000C0FF370010C0B3007A6002000000000025
:1096F00010C0B300DC5A020000000000B9FF3700C0
:10970000C85A0200000000004804DD00C85A0200E8
:10971000000000000080FB0080057400C85A0200B1
:10972000000000004804DD00C85A020000000000EC
:109730000080FB000006740000002100808F5500AF
:1097400002003E00800F5600AF0036000040EB00E4
:10975000DC5A020000000000A2FF37008004EB008A
:10976000ED8020001D844400C85A02000000000063
:10977000004C78008904E800898F5500F9FF3A0011
:109780001C5F0200000000000B00E0000D00320032
:109790000004EB0070408000684078000080FB000F
:1097A000CC5F0200000000005660020000000000D4
:1097B000E14F5000E5FF32000804E800888F5500B3
:1097C000F4FF3A008C05E9000C00E00012003200C2
:1097D0008004EB00ED8020001D8444001460020032
:1097E00000000000004C78008B8F54000400310012
:1097F0000040EB007A600200000000000300370028
:1098000010C0B3007A600200000000008904E80084
:10981000890F5600F0FF3A00505F02000000000080
:1098200010C0B300DC5A0200000000000C00E00091
:109830006CFF32000004EB0070408000684078004C
:10984000DC5A0200000000000804E800880F5600FF
:1098500064FF3200F8FF370010C0B300DC5A02008A
:109860000000000022C2BF000008A300FDFF32007C
:109870003011800080407800004D7800E24F5000A9
:109880001700320005003E000004E0000C0032002A
:10989000E14F500008003A000D003700F04F500033
:1098A0001600320000C2B30080CF50001700320013
:1098B000E3CF50000E0032001000200018003700E7
:1098C00004560200000000001000200014003700C1
:1098D000E8550200000000001000200010003700D2
:1098E000D055020000000000100020000C003700DE
:1098F000205602000000000009003700C0CFB3006E
:109900001E4F600010002000050037001E40780048
:109910000014A1000004A000004F780010002000F7
:10992000DC5A0200000000002EFF37000040EB0070
:1099300087FE070010C0B300DC5A020000000000E0
:1099400028FF37000040EB00DC5A02000000000056
:1099500024FF37006FC06100004DE80010C0B30065
:10996000DC5A020000000000A0AF20000048EB001D
:109970001A04E0001BFF320000047800C9AF200089
:10998000C85A0200000000000080FB00CC5F02000B
:10999000000000005660020000000000DC5A0200D7
:1099A000000000001840E800004C7800994F50007B
:1099B0000CFF3100F2FF3700E3C06100014D780079
:1099C00020C0B300AA5E02000000000010C0B30077
:1099D000DC5A02000000000002FF3700034078005C
:1099E000A07702000000000010C0B300DC5A0200A3
:1099F00000000000FBFE37000040EB00DC5A0200D4
:109A000000000000F7FE37000B00E0005CFF3200B2
:109A100052FF37004F0778004F06BE004F05BE00CB
:109A20004F04BE000000060000C0EB00FA75020003
:109A3000000000000080FB0000000600FA75020034
:109A400000000000001020000000060010C0B3005D
:109A5000B0750200000000000080FB00000006005E
:109A600020B0200010407800B07502000000000017
:109A70000000060020B020001080FB00000006005F
:109A800020B020000048EB0041022000B000200080
:109A9000F4730200000000000000060011C0B300D3
:109AA00020B020000148780041022000B0002000D2
:109AB000F47302000000000000000600A0AE2000C9
:109AC0001044A00040B120000048EB00C922A800CB
:109AD000CB22A90000000600889FBE008A1F7800E4
:109AE000800078000004E90010032000800F54007B
:109AF00030003E0040B120001080FB00800F540079
:109B00000500390091022000F0022000F4730200E9
:109B1000000000000E013700E10020008005200059
:109B20009A730200000000000840E8002C5902006F
:109B300000000000408B2800505702000000000089
:109B40008040EB00E0B02000014878000140780040
:109B5000C344DD005AB12000E8B020000080FB00C3
:109B60000900400060407D000080FB00947202000C
:109B70000000000000C2B300DC5A02000000000038
:109B80001880FB000900400060407D00FA7502006B
:109B9000000000001840E800004C7800E74F50003B
:109BA000EEFF3600708B28006857020000000000AE
:109BB000E700370050052000808F5000CE003200B3
:109BC00006003E000100E0000E00320030032000DD
:109BD000808F5000DA003A00A4003700C00E200049
:109BE000808F50004800320064004000808F500099
:109BF00045003200C00C2000808F5000D0003A0099
:109C0000C6003700D100200060062000F473020077
:109C1000000000007101200030072000F4730200F2
:109C20000000000040B120001004E00005003A00F0
:109C300091022000F0022000F473020000000000F6
:109C40002C003700F0B020000048EB0080047800C2
:109C5000E8B020005AB1200000C2B300DC5A020074
:109C6000000000001940E8002C590200000000002C
:109C7000808B280050570200000000000040EB00DD
:109C8000004C78000080FB009980FB00C308DD00D9
:109C90000100400060407D000080FB0094720200E3
:109CA0000000000000C2B300DC5A02000000000007
:109CB0001840E800004C7800E74F5000F1FF3600F4
:109CC00061002000A00820009A730200000000003C
:109CD0001980FB004300DD0060407D00C8000700E4
:109CE0009940E800814C780040B1200090CF5000AE
:109CF000D9FF3900310D200000092000F473020063
:109D00000000000092003700A08220000148780087
:109D1000C00E2000808F500005003A003101200065
:109D200030162000F4730200000000000400370029
:109D3000D100200060172000F47302000000000032
:109D40007101200030072000F473020000000000C1
:109D50000044EB00E0B0200008487800D70007007E
:109D6000F1B020008048780041B120008848780098
:109D70000004E00038003200EAB020008004EB006C
:109D800058B6200000C2B300DC5A020000000000F8
:109D90001A40E8002C59020000000000808B2800C7
:109DA0005057020000000000695888000900780040
:109DB00060407C000080FB00947202000000000004
:109DC00000C2B300DC5A02000000000060588000AE
:109DD0000000E80060588800E70F5000F4FF3600EC
:109DE00061002000A00820009A730200000000001B
:109DF00018407800820007009A427800E9CF5200AC
:109E00000F003E00695888008900780042B12000A8
:109E100054B1200053B620001280FB004300DD0047
:109E20000100400061C3790006707A008100E800FB
:109E3000E88F5000F8FF3A00615888001249E800A6
:109E4000054DE800A7000700F1B020008048780029
:109E50000004E000CBFF3A00B102200030182000DF
:109E6000F4730200000000003900370040000700D2
:109E700011012000E01A20009A7302000000000087
:109E800030C3B300FA750200000000000000EB00D0
:109E9000605888000004780039B0200000C0EB0052
:109EA000FA7502000000000000F47C006058800099
:109EB00060C07C000080FB00947202000000000083
:109EC00000C2B300DC5A02000000000060588000AD
:109ED0000004E80068588800E70F5400EFFF3600E0
:109EE000708B2800685702000000000019407800BD
:109EF00043000700160037001D0007000101200085
:109F0000F01B2000F47302000000000050C5B300F5
:109F1000FA750200000000000D0037001400070071
:109F2000F1002000F01C2000F4730200000000008B
:109F3000C0CCB300FA750200000000000400370036
:109F400041022000E01D2000F47302000000000028
:109F50004F0578004F04BE0000000600910020006D
:109F6000200A2100F4730200000000000000060037
:109F7000881F78007475020000000000004478001B
:109F8000A1002000202020009A73020000000000A1
:109F90000804E00005003A003100200080BB2000EA
:109FA000F47302000000000013003700910020004D
:109FB000C02020009A730200000000000808A300DF
:109FC0000400320051012000502120009A73020049
:109FD000000000000818A300040032004101200026
:109FE000A02220009A73020000000000708B28005D
:109FF00068570200000000004F04780000000600CF
:10A000008040780020C2B30080CF5000170032009B
:10A0100005003E00E4CF500019003200F0CF5000A0
:10A0200021003A000700370080C2B30080CF500003
:10A03000090032006540400080CF50001A003A000D
:10A0400014003700B1012000E0232000F473020067
:10A050000000000018003700A1012000902520001A
:10A06000F4730200000000001300370051012000CB
:10A0700030272000F4730200000000000E003700BB
:10A080008101200080282000F473020000000000FD
:10A090000900370001012000002A2000F4730200AB
:10A0A0000000000004003700E1002000002B200029
:10A0B0009A73020000000000000006008040EB00E0
:10A0C000D0B6200001487800F0B6200001487800A2
:10A0D000E0B6200001487800050007000080FB0082
:10A0E00000000600020007000080FB0000000600E0
:10A0F000889FBE008A9FBE008C9FBE000044EB007C
:10A1000000B7200008487800F9B620001904E000E4
:10A1100067003A0074750200000000000004E000CF
:10A1200007003200D0B6200008487800884C78003C
:10A13000E0B62000084878000000EB00640037001B
:10A14000A082200010407800FA7502000000000094
:10A150001BC0B3008046EB000D4578008B447800AF
:10A160005CB6200010C0B300B07502000000000013
:10A170000044780010C0B300B07502000000000079
:10A18000E14F540003003A00E14F50001D003A0037
:10A1900036003700804F54000200320088417800BA
:10A1A00020003700D0B620001040780080CF550046
:10A1B000060031000A80FB0060407E0080C1640020
:10A1C0000600320013C0B3000400370000C06D0069
:10A1D0000080FB000000E900CF01DE000304E00086
:10A1E00006003A00E8CF55000C003E00E0B6200023
:10A1F0000B4878008B4678000A003700E1CF510009
:10A2000008003A008A80FB0061407E0000C07400B4
:10A2100080707E0013C0B300070037008B467800C3
:10A220008041EB000A80FB0089C0EA0060417E00AB
:10A2300082C0600001707E0003407800B0750200AB
:10A24000000000008B45E80089C4440005003A0086
:10A250000A80FB0060407E00570007000A45E800C6
:10A2600019C0B300E74F5500BEFF360000C4B3006D
:10A2700080CF55000E00360000B720001004E0002B
:10A280000B003A00D0B620000D4878000D04E00025
:10A2900003003A0011C0B300F0B620000148780076
:10A2A00011C0B30050B620001004E00007003A00CF
:10A2B0008040EB00D0B6200001487800F0B62000C6
:10A2C00001487800E0B62000014878000180FB00DA
:10A2D0004F06BE004F05BE004F04BE000000060042
:10A2E0000800FA00889FBE008A1F78000000EB007B
:10A2F00051B62000E0C178006E81570003717800EC
:10A300000000E800E80F5000FAFF3A00D2B6200043
:10A3100012457800F1B6200091447800E0B62000A4
:10A320001044780000C4B300004978008048EB0076
:10A330006FFF07000004E0000C0032000001EB009A
:10A3400053B620006E805700E040790062C079006B
:10A3500080CF500005003A000201E800E80F5100EC
:10A36000F8FF3A0012C0B300010037000041EB00D3
:10A370000000EB0051B62000EE815700E37078003A
:10A380000000E800E80F5000FBFF3A00D0B62000C4
:10A390000A487800F0B6200009487800E0B62000AE
:10A3A000084878000280FB004F0578004F04BE008B
:10A3B0000080FA000000060002B72000124068008A
:10A3C0000080FB00B182200060C078000049780066
:10A3D0000080FB0000000600A08B28005057020000
:10A3E0000000000000000600889FBE008A9FBE009B
:10A3F0008C1F7800C922A800CB22A900C8C2A900DE
:10A40000A1AE2000114078000034A1000044A0005B
:10A4100080487800F0FF07003AB120000CB120001E
:10A42000C85A02000000000080417800004D78000A
:10A430000080FB004400DE0021B12000804878004D
:10A44000E14F50005300320003003900E44F500048
:10A450006E003A0066003700E2CF51000F00320074
:10A4600005003E000304E0006C003200E1CF510023
:10A4700044003A0007003700E4CF51000E003200DC
:10A480004000390068C05100E14F50003D003E00DF
:10A490000F003700D0FF0700E1FF3700747502009E
:10A4A00000000000004E780010C0B300DC5A02002B
:10A4B00000000000DAFF370000C0EB00FA75020070
:10A4C00000000000DC5A020000000000D4FF37004A
:10A4D00010C0B300DC5A02000000000090C0B300BE
:10A4E0009A4F100004003A00C1CEB300A0822000B1
:10A4F000014878000300370001CFB300A08220009C
:10A5000001487800EDFE0700004E78000004E000EE
:10A510001100320018B120008045EB0059B6200030
:10A520000B4C78000B4078000080FB0060C07C0082
:10A53000DC5A0200000000001840E800004C7800DF
:10A54000E74F5000F8FF3600E6FE0700004E7800A7
:10A550000004E000F2FF3A0010B120000048EB00D8
:10A560000004780000C0EB00DC5A0200000000008C
:10A570001840E800004C7800E74F5000A8FF3E006C
:10A58000F8FF37000040EB00DC5A0200000000003A
:10A59000A3FF37006FC06100004DE80010C0B3009A
:10A5A000DC5A02000000000010B120000048EB005F
:10A5B0001A04E0009AFF32000004780039B120004C
:10A5C000C85A020000000000FA75020000000000F6
:10A5D00010C0B300DC5A0200000000001840E80080
:10A5E000004C7800994F50008DFF3100F4FF370088
:10A5F00003407800A07702000000000010C0B30004
:10A60000DC5A02000000000085FF37000040EB002C
:10A61000DC5A02000000000081FF37004F0678007E
:10A620004F05BE004F04BE00000006000000EB0016
:10A6300080088800F0088800E00C8800E25B800059
:10A640000200E00006003A00CAC6BF0001CEB30017
:10A6500001406000CAE6B700925B88002E00370018
:10A66000E30F510004003C0010A1A8001081A800D5
:10A67000E003200010003700FE0F510004003C00F2
:10A6800010A1A8001081A900A00F20000A00370027
:10A69000400F2000800F510004003C0010A1A900D1
:10A6A0001081A800007D20000300370010A1A90040
:10A6B0001081A90000E82300110009000280D800E1
:10A6C0000000E90060088800F25B80000280B900A9
:10A6D00042062000110009000280D800A26C200070
:10A6E0001241780003CEB300034161006241B30020
:10A6F0000001FD00CAE6B7000001FD00D00C880093
:10A70000C00C880060002000E00C880011E1A80067
:10A7100020002000905B880000000600889FBE009B
:10A720008A9FBE008C1F78000004EB008808880018
:10A73000F8088800E80C8800905B8000E20F500069
:10A7400010003A00CAC6BF0001CEB300014060004D
:10A75000CAE6B700C1002000E02B2000F47302001D
:10A7600000000000985B8800106480000000E80092
:10A770000080FB0001B8200060C078000004E00009
:10A780008B003200106480000000E8000080FB00B5
:10A7900010648800EA19020000000000541802004A
:10A7A0000000000000047800EA1902000000000028
:10A7B0005418020000000000CF80DE00E803020011
:10A7C000000000000005BE000001EB008800E90069
:10A7D000E0F92000808F500001003E0012002000B0
:10A7E000820478006011B8000A00BE003E04020036
:10A7F000000000000000E00008003400020020001B
:10A80000832C24000A00BE00420402000000000065
:10A810000000E00001003D008904E800E28F5400E0
:10A82000110032000004EB002864880011012000B0
:10A83000A02C2000F4730200000000001101200091
:10A84000B02D20009A7302000000000088017800FB
:10A8500002FA20001100200020032000E41A020068
:10A860000000000000047800E30F540004003E00E4
:10A8700010A1A8001081A800E003200010003700FC
:10A88000FE0F540004003E0010A1A8001081A90092
:10A89000A00F20000A003700400F2000800F540056
:10A8A00004003E0010A1A9001081A800007D200036
:10A8B0000300370010A1A9001081A90000E82300BF
:10A8C000110009000880D8000006E900E28F54005A
:10A8D0000E00320001012000902F20009A73020028
:10A8E000000000008001EB003206200083007800A9
:10A8F00020032000E41A020000000000CF80DE00E8
:10A90000E8030200000000000005BE000200200075
:10A91000832C24000A00BE00460402000000000050
:10A920000004BE006160B900E803020000000000FE
:10A930000C00E00004003D00020020000378240029
:10A94000CC040200000000000001BE000800BE00B0
:10A950008605020000000000EE0502000000000075
:10A96000A26C20001241780003CEB30003416100C5
:10A970006241B3000001FD00CAE6B7000001FD001E
:10A98000D00C8800C00C880060002000E00C88001B
:10A990006C08880011E1A800A10020009030200080
:10A9A000F47302000000000020002000905B88008B
:10A9B0004F0678004F05BE004F04BE0000000600A1
:10A9C000905B8000E20F500005003A00F10120008A
:10A9D00030312000F4730200000000002D00370029
:10A9E000F1002000203320009A73020000000000D4
:10A9F0000000EB00F008880080088800C942A80029
:10AA000086C6BF0001CEB30001406000A040B30085
:10AA100086E6B700A0032000800888003E000700FB
:10AA2000F20F2000820F5000E08F58000500360022
:10AA3000C808DD000080FD00804078000040EB0089
:10AA400007003700B1002000A01321009A73020014
:10AA500000000000A0002000800888002E000700F1
:10AA60001858020000000000208D280050570200F6
:10AA700000000000608D2800685702000000000000
:10AA8000F0C1B3008666B7000000EB00F008880054
:10AA900080088800000006000000EB00F008880035
:10AAA00080088800C942A80086C6BF0001CEB30056
:10AAB00001406000A040B30086E6B700A00320007C
:10AAC0008008880014000700F20F2000820F500059
:10AAD000E08F5800050036004809DD00C801DE009F
:10AAE000830171004801DD0004003700A000200050
:10AAF00080088800080007000001BE00F0C1B30014
:10AB00008666B7000000EB00F00888008008880027
:10AB10000200BE00000006000080EB007008880004
:10AB2000600888000000EB004008880030088800BA
:10AB3000B0088800A008880080002000F008880085
:10AB4000400F2000E008880000402200D008880064
:10AB50008780A9001FE1A80011E1A80087C0BF00FD
:10AB60000048A300FDFF320011E1A9001FE1A90088
:10AB700030088000D05B880042088000C25B8800FB
:10AB800003002000C011DD00020020000000410091
:10AB9000E0804900A05B8800B15B880000000600EF
:10ABA000A0AE2000104078006340600002003A0030
:10ABB000C942A80001003700C8C2A800E100200077
:10ABC000103420009A73020000000000000006000C
:10ABD000A0AE2000104078006340600003003A00FF
:10ABE000C942A900CB42A80002003700C8C2A90090
:10ABF000CAC2A80081002000F0342000F4730200D3
:10AC00000000000000000600A0AE20001040780008
:10AC10006340600003003A00C942A900CB42A9008A
:10AC200002003700C8C2A900CAC2A90071002000F2
:10AC300070352000F47302000000000000000600E0
:10AC4000A0AE2000104078006340600007003A008A
:10AC5000C942A8000000000000000000CBC2BF00F5
:10AC60004200DE006140600006003700C8C2A80054
:10AC70000000000000000000CAC2BF004600DE0065
:10AC8000614060000080FB0000000600889FBE005D
:10AC90008A1F78000004EB0088088800F808880004
:10ACA000E80C8800905B8000E20F500011003A0031
:10ACB000106480000000E8000080FB0001B8200064
:10ACC00060C078000004E0000A003A00CAC6BF0075
:10ACD00001CEB30001406000CAE6B700C100200009
:10ACE000E02B2000F473020000000000985B880055
:10ACF00060003700106480000000E8000080FB0066
:10AD000010648800EA1902000000000054180200D4
:10AD100000000000CF80DE00E80302000000000019
:10AD20000004BE002A6480000A00E00006003A0029
:10AD300002002000433324003E0402000000000013
:10AD40000000E000110034000004EB0028648800DB
:10AD500031012000301E2100F473020000000000C9
:10AD600088017800420B200088007800A0052000B0
:10AD7000E41A020000000000CF80DE00E8030200B9
:10AD8000000000000004BE001AC0B30010A1A8001B
:10AD90001081A80002002C00A35524000800BE006A
:10ADA000460402000000000002002400C349240001
:10ADB0008605020000000000020020008327240016
:10ADC000CC04020000000000EE05020000000000BC
:10ADD000A26C20001241780003CEB3000341610051
:10ADE0006241B3000001FD00CAE6B7000001FD00AA
:10ADF000D00C8800C00C880060002000E00C8800A7
:10AE0000204E20006008880011E1A800C100200049
:10AE1000601F2100F47302000000000020002000E9
:10AE2000905B8800E14F550012003A0013002000AB
:10AE3000420B20008000EB000080EB00E41A0200CF
:10AE400000000000CF80DE00E803020000000000E8
:10AE50000004BE006011B8004204020000000000BF
:10AE60000000E000C9FF3D00608D28006857020027
:10AE7000000000004F0578004F04BE0000000600EF
:10AE80000000E0000300320010C3B300CA01070055
:10AE90000200370000C3B300C7010700000006002E
:10AEA000881F7800B0407800000478000104E000BA
:10AEB0000500320001407800BF010700B84078006B
:10AEC0000104E000FBFF3A004F0478000000060098
:10AED000881F7800B0407800000478000104E0008A
:10AEE0000500320001407800B3010700B840780047
:10AEF0000104E000FBFF3A00D0C0B300AE01070040
:10AF0000A0C0B300AC0107004F04780000000600A9
:10AF1000889FBE008A1F78000045780000872800BF
:10AF2000DFFF070009C8B30088C0B300094065000F
:10AF30000300320010C3B3009F0107000200370076
:10AF400000C3B3009C0107000980FB008004D1000E
:10AF50000844E900F5FF3A004F0578004F04BE00B1
:10AF600000000600E4874700889FBE008A9FBE005D
:10AF70008C9FBE008E1F78000006BE000040EB00D4
:10AF800080F79F000A102E005B5F20008EC0B30088
:10AF90000A01BE000C00BE002406020000000000F2
:10AFA0000004BE008FF097000104E00003003A00A7
:10AFB000E00F5400E08F5C000C00320001C3B300CE
:10AFC000014044007C0107000851B8000BC0B900E3
:10AFD0000300400009D2B900840140000206560077
:10AFE00083865E0010C0B30080F79F00A20020009F
:10AFF000030020000A00BE0024060200000000003A
:10B000000005BE000E47E900E1FF3A0001C3B300AE
:10B0100001404600680107004F0778004F06BE0058
:10B020004F05BE004F04BE004F00B10000000600F7
:10B03000889FBE008A9FBE008C1F78000004BE005F
:10B04000F0232400F1002000800F5400818F5C0069
:10B050001700360002242400F30020000800BE0080
:10B06000240602000000000056000700C0C2B30022
:10B070005101070002242400F30020000800BE0054
:10B0800044060200000000000004BE001C00200076
:10B09000703E2000800F5400E08F5C000A003E00EC
:10B0A000308728007EFF0700100020002B003700AB
:10B0B0000000EB00713E2000810F5400E08F5C0027
:10B0C000260036000006EB00823E20000300200030
:10B0D0000800BE0024060200000000000005BE00BB
:10B0E00040062000800F5500E08F5D000300360011
:10B0F0000A007800330007000F0037000C00E00062
:10B100000B003200EA0F5500E08F5D0003003600AF
:10B1100000C3B30028010700020037008087280021
:10B120005FFF07000A0078002600070002003700D2
:10B130000A00780023000700C0C2B3001E01070008
:10B14000823E2000030020000800BE0044060200EA
:10B15000000000000004BE00100020004106200096
:10B16000810F5400E08F5C00030036000800780077
:10B17000140007000F0037000000E0000B00320051
:10B18000EA0F5400E08F5C000300360000C3B300F8
:10B1900009010700020037008087280040FF0700F0
:10B1A0000800780007000700020037000800780058
:10B1B000040007004F0678004F05BE004F04BE0094
:10B1C00000000600889FBE008A9FBE008C1F78008A
:10B1D000800478008040EB000A7122004BC0B3006D
:10B1E000AC002000811F7800110009008A84D8007B
:10B1F00000047800CF0078000104E00002003A006B
:10B200000800E0000600320001C3B3000140440022
:10B21000E90007000AC0B9008084540011C0B300DF
:10B22000811F7800110009000C85D8000005780006
:10B23000CF0078008B45E900EAFF3A0001C3B30074
:10B2400001C04400DC0007004F0678004F05BE0037
:10B250004F04BE0000000600889FBE008A9FBE000B
:10B26000804478008041EB004AC6B3002BC0B30095
:10B270000980FB000A81FB00110009000280D80050
:10B280008000FD00014478000304E00002003A0061
:10B290000104E0000600320001C3B3000140440095
:10B2A000C50007000AC0B90080C4540013C0B30031
:10B2B0000A80FB00A2002000110009000280D800D3
:10B2C000004578008B45E900E9FF3A0001C3B3006F
:10B2D00001C04400B80007004F05BE004F04BE0087
:10B2E00000000600889FBE0080047800B088280017
:10B2F000EBFE07004448DE006F006000B8872800BE
:10B3000060407C00AC0007006F80640060407C00FF
:10B31000A90007004F04BE0000000600889FBE0081
:10B320008004780000C3B3008500070080C7B30025
:10B33000830007004448DE006F006000B8872800E3
:10B3400060407C007E0007006F80640060407C00ED
:10B350007B0007004F04BE0000000600889FBE006F
:10B3600080047800B0882800CDFE07004C48DE003D
:10B37000B887280060407C008F0007004848DE0046
:10B380006F00600060407C008B0007004448DE00D6
:10B390006F00600060407C00870007006F806400E1
:10B3A00060407C00840007004F04BE0000000600DF
:10B3B000881F78007D00B900D2022000110009002A
:10B3C0000280D8008000FD00420620001100090024
:10B3D0008280D800010478009FFF0700E0C2B3001C
:10B3E00075000700E94F540002003E0000C3B3009F
:10B3F000710007000840780097FF07004F047800AD
:10B4000000000600220320001241780032E0B7005D
:10B410001180BA009100BA000001FD0032E0B700CF
:10B420000001FD004800DD00010070000000060082
:10B430000081200010407800E94F500005003200E4
:10B440000080FB0000004000C1A92000E0807800DF
:10B45000411188000000EB00001188002062A80064
:10B460001011880021E2A8002342A8008560A900ED
:10B470000000060023C2BF000000D1006100600090
:10B480000000060022C2BF0061006000000006004C
:10B490000000EB005069880010002000406988001F
:10B4A000A081200010A0A1000000060023C2BF0060
:10B4B0000018A3000E003A00506980008000E800E8
:10B4C00000002100808F500001003A008000EB0056
:10B4D00040698000808F500005003200516988006B
:10B4E00070408000614078000080FB0020118800DF
:10B4F00000000600426980007440800003002100C3
:10B50000506980008000E800838F500001003A00FD
:10B510008000EB00828F50000800320023C2BF0081
:10B520000018A300F6FF3A005169880061407A00D4
:10B530000080FB0020118800F1FF370000000600AA
:10B54000004178004169800050698000808F500080
:10B5500004003A00C222A900A081200010A0A0008F
:10B560000A003700704080008270780040698000D7
:10B570000000E8004069880001002100810F5000B0
:10B5800002003A000000EB0040698800000006005D
:10B5900022C2BF000008A300FDFF3200301180006E
:10B5A0000080FB000000060023C2BF000008A300CB
:10B5B000FDFF32000000060000417800A18120005C
:10B5C000001020001100600005003A0023C2BF00F7
:10B5D0000018A300FDFF3A000200FB0020118800C4
:10B5E000000006000080FB004011880000000600FB
:10B5F00022C2BF000000D100610060000000060010
:10B600002222A9000000060095C0BF000048A30048
:10B610000D003A004140800050408000810F5000F2
:10B620000900320023C2BF000018A300FDFF3A004A
:10B630008580A9009580A800304080006140780096
:10B640000080FB002011880000000600809FBE00E3
:10B65000821F78003211800021408000004080006D
:10B6600082707800204080000000E80020408800C0
:10B6700011408000810F500001003A009560A90040
:10B680008560A9004F0178004F00BE000040060011
:10B69000809FBE00404080008000E800414088005C
:10B6A00050408000808F500002003A009580A90031
:10B6B0000400370030408000614078000080FB00CB
:10B6C000201188008580A9004F00BE0000400600C0
:10B6D000808D280050570200000000000000060086
:10B6E000889FBE00C222A800D8000700F8FF07000C
:10B6F000D20007008040780000D420000148780084
:10B700000104E000C800350002003A00F0FF070025
:10B71000F7FF3700E1CF500006003A00CB000700EA
:10B720000E34020000000000C8000700E8FF070018
:10B73000EFFF3700E2CF500006003A00C3000700D9
:10B74000C84A020000000000C0000700E0FF070038
:10B75000E7FF3700E3CF500006003A00BB000700C8
:10B76000C63C020000000000B8000700D8FF070038
:10B77000DFFF3700E4CF500006003A00B3000700B7
:10B78000F451020000000000B0000700D0FF0700E5
:10B79000D7FF3700E5CF500006003A00AB000700A6
:10B7A0001C3F020000000000A8000700C8FF0700BF
:10B7B000CFFF3700E6CF500006003A00A300070095
:10B7C000A06D020000000000A0000700C0FF0700FD
:10B7D000C7FF3700E7CF500004003A009B00070086
:10B7E0009A000700BAFF0700C1FF3700EFCF5000F3
:10B7F00008003A0010C0B300DC5A0200000000004C
:10B80000C222A900D45A0200000000000000FE007D
:10B81000B7FF3700F0CF500003003A000040EB00C4
:10B8200019010700B2FF3700F1CF500003003A00C2
:10B8300010C0B30014010700ADFF3700F2CF500075
:10B8400025003A000000EB0080088800F00888001E
:10B85000E00C8800CAC6BF0001CEB3000140600002
:10B860006041B300CAE6B700740007000080FB0027
:10B870000018A3000100320010A1A8000008A300D6
:10B88000010032001081A8006C0007004804DD00B0
:10B890006A0007000080FB0000007400D00C8800E4
:10B8A000C00C880060002000E00C880063000700E6
:10B8B0004804DD00610007000080FB000000740008
:10B8C0006008880011E1A80010C0B300DC5A020033
:10B8D0000000000086FF3700F3CF50000B003A0055
:10B8E0000000EB0080088800E00C8800CAC6BF009A
:10B8F00001CEB30001406000CAE6B70010C0B3003B
:10B90000DC5A02000000000079FF3700F4CF50003D
:10B910000D003A0021E3A800C0C0B3001672020077
:10B92000000000000004780021E3A9004800DE00C8
:10B93000DC5A02000000000008407800DC5A0200D7
:10B94000000000006AFF3700F5CF500015003A00F4
:10B9500021E3A800C0C0B30016720200000000007E
:10B9600000047800D45A0200000000004840DE00C5
:10B97000DC5A02000000000008407800DC5A020097
:10B9800000000000425A020000000000E14F500099
:10B99000F0FF3A00C85A02000000000021E3A900AD
:10B9A00053FF3700F6CF500014003A004C55020008
:10B9B000000000000004BE004808DE00DC5A02005F
:10B9C000000000004048DE0001002000DC5A0200B8
:10B9D000000000004849DD004840DE000000710022
:10B9E000C848DE00DC5A0200000000000840780071
:10B9F000DC5A0200000000003DFF37000168A30090
:10BA0000050032000140780015000700DC5A0200F2
:10BA10000000000036FF37000040EB00DC5A020057
:10BA20000000000032FF3700014078004A000700A4
:10BA3000DC5A0200000000002DFF3700C85A020047
:10BA4000000000000080FB000000060000C0EB00CA
:10BA5000030007000040EB003F0007000000060065
:10BA6000881F7800004478000081FB00C410DE00CD
:10BA7000E1C06000C208DD00C9C2BF000024A1000F
:10BA800001407000C9E2B700C310DE00E1C06000F1
:10BA900081C04000C9C2BF000014A1000140700075
:10BAA000C9E2B700C210DE00E1C06000C9C2BF0039
:10BAB0000004A10001407000C9E2B7000201D100FA
:10BAC0004711DD00C8C2BF000074A1000240700031
:10BAD000C8E2B700E1406400C608DD00C8C2BF008C
:10BAE0000064A10001407000C8E2B70050002000CF
:10BAF000447302000000000000CEB30080406400E8
:10BB0000CBC2BF000028A300010032000144A00006
:10BB1000CBC2BF000018A300010032000134A00016
:10BB2000CBC2BF000008A300010032000124A00026
:10BB3000CA42E20001003D000114A000CAC2BF00D9
:10BB40000068A300010032000104A0000180FB0096
:10BB50004F04780000000600881F78000044780039
:10BB60000081FB000268A30003003200C002A900AC
:10BB7000C202A80002003700C002A900C202A90048
:10BB80000258A30003003200C962A800CB62A900DA
:10BB900002003700CB62A900C962A900C410DE0010
:10BBA000E1C06000C208DD00CBC2BF000024A100DC
:10BBB00001407000CBE2B700C310DE00E1C06000BE
:10BBC00081C04000CBC2BF000014A1000140700042
:10BBD000CBE2B700C210DE00E1C06000CBC2BF0004
:10BBE0000004A10001407000CBE2B7008200D10048
:10BBF000C708DD00CAC2BF000074A1000140700088
:10BC0000CAE2B700E1406400C608DD00CAC2BF0056
:10BC10000064A10001407000CAE2B700500020009B
:10BC2000447302000000000000CEB30080406400B6
:10BC3000CBC2BF000028A300010032000144A000D5
:10BC4000CBC2BF000018A300010032000134A000E5
:10BC5000CBC2BF000008A300010032000124A000F5
:10BC6000CA42E20001003D000114A000CAC2BF00A8
:10BC70000068A300010032000104A0000180FB0065
:10BC80004F04780000000600881F7800804078008C
:10BC90000040EB004C6B0200000000000044780004
:10BCA0000004E00001003200C222A8000840780031
:10BCB000DC5A020000000000425A020000000000AE
:10BCC0000004E0000D003200C85A0200000000002D
:10BCD000E14F40000400320000404400DC5A020002
:10BCE000000000000500370010C0B300DC5A02005D
:10BCF000000000004F047800000006000804E00087
:10BD0000EDFF3A00106A80000000E0000D003A00EC
:10BD10000080EB00106A8800C2C2BF000000D100A2
:10BD2000610060000004A20000404000212C2000BF
:10BD3000914078000114A10080C0700001007800DB
:10BD4000C2E2B700106A80000000E900106A8800B3
:10BD5000D9FF37000141780061D320008048780086
:10BD6000E34F500005003A0000202000C069880021
:10BD700000082000D0698800030037000020200060
:10BD8000C0698800D0698800E14F51000E00320080
:10BD900003003900E24F51001F003A001400370041
:10BDA00041C1B300C0D320000148780041C6B300B0
:10BDB000D0D320000148780021C3B300E0D3200095
:10BDC000014878001B00370021C0B300C0D3200019
:10BDD00001487800A1C0B300D0D32000014878000A
:10BDE00051C0B300E0D320000148780011003700B3
:10BDF00011C0B300C0D320000148780051C0B30087
:10BE0000D0D320000148780021C0B300E0D3200047
:10BE100001487800070037008040EB00C0D32000C5
:10BE200001487800D0D3200001487800E0D32000FA
:10BE30000148780000000600889FBE00D0D3200093
:10BE40009040780000302000E2000700CBC2BF0025
:10BE50000008A30004003200CBC2BF008004EB0046
:10BE60000018A30001003A0019002000D8D32000D8
:10BE70009840780000202000E600070098407800F5
:10BE800000102000E3000700984078000020200008
:10BE9000D0000700090078004F04BE000000060033
:10BEA000881F7800D8D32000984078000030200008
:10BEB000D80007009840780000102000C500070057
:10BEC0009840780000202000C20007000000EB002E
:10BED0004F04780000000600889FBE008A9FBE00C5
:10BEE0008C9FBE008E1F78008001780090AD2000EE
:10BEF000104178000280FB000000E90011002000E2
:10BF0000800EDD008005EB000204E0001C00320022
:10BF1000830478000005EB008A057800CED320006A
:10BF2000DCD320000D8064001E4178000120200039
:10BF3000BF0007009C40780000102000A50007000B
:10BF400000082000CF000700004478009C407800E3
:10BF500000102000AF000700898444008B85450055
:10BF60000804E000010032008B05E8000A05E80043
:10BF700090AD20001080FB008A0F5000E9FF3E00CA
:10BF80000B0078004F0778004F06BE004F05BE003B
:10BF90004F04BE0000000600889FBE008A9FBE00BE
:10BFA0008C1F78008001780090AD2000104178004F
:10BFB0000280FB000000E90011002000800DDD0080
:10BFC0000204E00014003200030478008004EB0057
:10BFD000CCD32000DAD320000B0064001C41780091
:10BFE00001202000920007009A40780000102000F5
:10BFF000780007009A4078000010200085000700B4
:10C00000080444008904E80090AD20001080FB0083
:10C01000808F5400F0FF39004F0678004F05BE00B6
:10C020004F04BE0000000600889FBE008A9FBE002D
:10C0300000202000930007000005EB0090AD2000D9
:10C040001004E000150032008004EB0009057800C0
:10C05000DBD320009B407800001020005D0007002B
:10C060000020200087000700004478009B407800F3
:10C0700000102000670007000A0545000804E000E2
:10C08000010032000A05E8008904E80090AD2000B4
:10C090001080FB00890F5000EEFF3E000A00780080
:10C0A0004F05BE004F04BE0000000600889FBE0082
:10C0B000A8D320001800780072000700D9D3200010
:10C0C0009940780000102000420007001800780016
:10C0D0006C000700004478009940780000102000B0
:10C0E0004C0007000884FB00080078004F04BE00E5
:10C0F00000000600881F78000080FB00C1D32000EC
:10C1000011417800C169800049000700D8D32000A0
:10C1100098407800001020002E000700984078001A
:10C12000001020003B0007004F04780000000600CC
:10C13000889FBE008A1F7800804478000004E000D9
:10C140000B0032000044EB00DAD320009A40780064
:10C15000001020001F0007009A4078000010200007
:10C160002C0007000844E80088CF5400F7FF3A008D
:10C170004F0578004F04BE00000006000080FB0061
:10C18000C1D3200011417800C16980002800070058
:10C19000000006000080FB00C1D3200011417800A0
:10C1A0000110200022000700000006000080FB00B4
:10C1B000C1D3200011417800010420001C000700B9
:10C1C00000000600D06980002E0007000080FB0000
:10C1D0000000060000017800A0AE200010407800AA
:10C1E0007040600005003A0002007800CC22B700E1
:10C1F0000280EA00C822B600020037000200780080
:10C20000C822B7000180FB00447302000000000058
:10C21000000006000080EA00CC22B600C822B6006A
:10C220000180FB00447302000000000000000600D3
:10C230000000E00004003A000180EA00CC22B600D1
:10C24000C822B6000B003700A0AE200010407800D6
:10C250007040600005003A0001007800CC22B70071
:10C260000180EA00C822B600020037000100780011
:10C27000C822B7000280FB004473020000000000E7
:10C2800000000600C822B700000000000000000007
:10C29000000000008000EB00CA02B600010032007E
:10C2A0001100200001007800000006001460020068
:10C2B0000000000000000600CC5F0200000000004B
:10C2C00000102000000006001C5F020000000000BB
:10C2D00081002000009320009A73020000000000FB
:10C2E000D1002000A0412000F473020000000000F3
:10C2F00000000600505F0200000000006100200006
:10C30000809320009A73020000000000C10020000A
:10C3100070422000F47302000000000000000600DC
:10C3200056600200000000000080FB0000000600D4
:10C33000E2600200000000000080FB000000060038
:10C340000040EB00CA600200000000000000060090
:10C3500010C0B300CA600200000000000000060028
:10C3600010C0B3009860020000000000000006004A
:10C370000040EB00BE60020000000000000006006C
:10C3800010C0B300BE600200000000000000060004
:10C3900001012000D09820009A73020000000000E4
:10C3A00080AD2000104078002C59020000000000F1
:10C3B00000C2B300DC5A020000000000A0AE200062
:10C3C0001080FB004400DE00614060002C59020038
:10C3D0000000000000C2B300DC5A020000000000B0
:10C3E0003100200020AE20009A73020000000000FF
:10C3F00000000600881F7800EA1902000000000013
:10C40000541802000000000000047800EA1902003D
:10C4100000000000541802000000000080007800B6
:10C420000800E900E30F5000020036000004EB00B2
:10C430000200370080AD20000848E9000100E90053
:10C44000E10F500008003E00A0AE2000E1C06000F7
:10C45000C408DD00104178000244A10001487100C9
:10C460000800E0001F003A000004EB002864880088
:10C47000B103200080452000F4730200000000009A
:10C4800088017800420020001100200010002000E8
:10C49000E41A02000000000081AD20008048E9009D
:10C4A000F1042000E0932000F4730200000000007B
:10C4B00088017800220020001100200010002000D8
:10C4C000E41A020000000000A2AE200061406000FB
:10C4D0004400DD00924078000144A10000C97000D2
:10C4E00001003700AAFF0700CB02A900CB22A90058
:10C4F000C922A800C902A90080AD200090407800A0
:10C5000020C0B300AA5E0200000000004F047800C3
:10C5100000000600E10F500009003200030039005E
:10C52000E20F500009003A000600370081032000A6
:10C53000D09920009A730200000000000700370025
:10C540000C0007001F000700040037004102200014
:10C55000E01D2000F473020000000000000006004F
:10C56000B1002000600B2100F47302000000000005
:10C5700000000600F1032000509D2000F47302002B
:10C58000000000000040EB00D66002000000000048
:10C59000F00F2000447302000000000010C0B30040
:10C5A000D66002000000000010C0B30098600200D6
:10C5B000000000000040EB00D66002000000000018
:10C5C000000006000400FA00889FBE00D10220008F
:10C5D00040A120009A730200000000006884570008
:10C5E000E48457001460020000000000005C780042
:10C5F0000080FB00725902000000000000C2B3007E
:10C60000DC5A020000000000888F5400F5FF3A0059
:10C61000C08E28006857020000000000A100200022
:10C6200010A420009A730200000000008FF8970009
:10C630000180FB004400DE00E94F50000E00320094
:10C6400003003E00E84F50001A003A000500370092
:10C65000EA4F50000D003200EF4F500015003A0035
:10C660000F00370061002000B0A420009A73020080
:10C6700000000000130037006100200010A520001A
:10C680009A730200000000000E00370061002000D5
:10C6900070A520009A730200000000000900370016
:10C6A00031002000D0A520009A7302000000000095
:10C6B000040037007100200000A620009A730200D9
:10C6C00000000000C08E2800685702000000000033
:10C6D000B100200070A620009A7302000000000044
:10C6E0001FFC97000878A30005003A0061002000B5
:10C6F00020A720009A730200000000000400370009
:10C70000F100200080A720009A73020000000000C2
:10C71000C08E28006857020000000000C100200001
:10C7200070A820009A730200000000000800780042
:10C730008007B2004380DE00004178000004E00082
:10C7400005003A00D100200030A920009A730200B1
:10C750000000000010003700000420008040EB00C3
:10C76000EF4F510005003A0031002000D0A5200015
:10C770009A7302000000000007003700000040002C
:10C780008140E800814F5100FCFF3A0082FF9F008A
:10C79000E258020000000000C08E28006857020026
:10C7A000000000009101200000AA20009A730200FE
:10C7B000000000001FF89700674160001000200093
:10C7C000060032008040EB00100020000000400016
:10C7D0008140E800814F5100FCFF3A002C590200D3
:10C7E00000000000C08E2800685702000000000012
:10C7F0004F04BE000080FA00000006000C08000094
:10C80000120000000200000000006C000D0000009B
:10C810000000000000000000000000000000000018
:10C82000D80A00001A000000000000006C0D000093
:10C830000010000000000000F20A000002000000EA
:10C84000000000001E0800000C00000002000000B4
:10C8500000181C001D0018001C1D03000B131B00FA
:10C86000F40A00000600000000000000FA0A0000C0
:10C8700008000000000000002A080000020100007B
:10C8800002000000F0005E00BCE261003FDD8300BA
:10C89000C29C7E0020A3FD001F419D00C3217F009C
:10C8A000FCA240001E5F0100E3BD3E006082DC0090
:10C8B000237D9F00C1421C00FEA0E100BF5D03007C
:10C8C00080DE3C0062BEE000025CDF0081633D0070
:10C8D0007C22C0009E1D4300A1FF460018FAA40060
:10C8E00027799B00C584DA003866E500BB5907004C
:10C8F000DB85670039BAE4000658190047A5FB003C
:10C900007826C4009A653B00D98704005AB8E6002F
:10C91000A7F91B0045C698007A24F800A6441A001F
:10C9200099C725007B3A640086D85B0005E7B9000B
:10C930008CD230006EEDB300510F4E0010F2AC00FF
:10C940002F719300CD114F00ADF370002ECC9200EB
:10C95000D38D6F0031B2EC000E50AF00F1134D00DB
:10C96000CE9072002C6D3300D18F0C0052B0EE00CF
:10C97000326C8E00D0530D00EFB1F000AE4C1200BF
:10C9800091CF2D0073CA94007628AB00F5174900AB
:10C990000856B400EA693700D58B570009EBB5009B
:10C9A00036688A00D495CB002977F400AA4816008F
:10C9B000E9B755000B88D600346A2B007597C9007B
:10C9C0004A14F600A8742A00C89615004BA9F7006F
:10C9D000B6E80A0054D789006B350000020B00004E
:10C9E0007000000000000000720B00000E0000004C
:10C9F000000000002C09000070010000020000008F
:10CA00003A773A00773A77003A77480077587700D4
:10CA10003A773A00773A77003A775800773A7700D2
:10CA2000587758007768770076778200778E77009E
:10CA300098774800695A00000000000000B84F00D5
:10CA4000B84F3A00773A77001E4D14004D3A770000
:10CA50003A774E004D404D003A4D30004D264D0086
:10CA600058776C004D5E4D008277AE004F9877008E
:10CA7000312D5700495245000000C6003AC63A0021
:10CA8000DA3ADA003A3E3700F0363A00773A770081
:10CA90003A773A00775877003A77580077EC3A00BF
:10CAA000B639D20037B03900583B460037554100FF
:10CAB00052540000000000007A477A0047CC47003B
:10CAC0003A77180047DA46003A773A00773A770023
:10CAD0003A775800773A77005877580077B048008F
:10CAE0002E48A200489E49000448490032430000F5
:10CAF0000000000000722E00502E94002E3A7700A5
:10CB0000BA2EB2002E3A77003A773A00773A770099
:10CB100058773A00775877005877E80030442F006C
:10CB2000E430A80031CE2E00535049000000000030
:10CB300000006400616461007A617A00615C6100F8
:10CB40005661A80061A06100C061B80061986100F1
:10CB5000B0619000615877008A62FA0061827700C4
:10CB6000B062C80061325700495245000000000021
:10CB70000A70D8006F3C70003C70C4006FBC6F003E
:10CB800086708E00709670009E707600707E7000C9
:10CB90006E70580077687700E670820077C0710089
:10CBA000A6703300574952004500000000F86800A5
:10CBB000F868060069066900E6685800773A770069
:10CBC0003A773A00773A770058773A007758770003
:10CBD00058775600691469002C328C006A987700E7
:10CBE0004C4344000000000000000000800B0000E7
:10CBF000A8010000000000009C0A000012000000D4
:10CC000002000000143404000D8206004003A0005E
:10CC100001CF00006700440000220000280D000042
:10CC20000400000000000000000800000C000000EC
:10CC300000000000AE0A0000280000000200000012
:10CC4000143404000D8206004003A00001CF000050
:10CC500067004400002200007F00140034040D002F
:10CC60008206400003A00100CF007F0000670000A3
:10CC700044002200000000002C0D0000080000000D
:10CC800000000000340D0000020000000000000061
:10CC9000360D00000A00000000000000400D0000FA
:10CCA0000400000000000000D60A0000020000009E
:10CCB0000200000003000000440D00000E00000010
:10CCC00000000000520D0000020000000000000003
:10CCD000540D00000200000000000000560D00008E
:10CCE000160000000000000000000000007C200092
:10CCF000C822B7000F00070020C0B30021000700C2
:10CD0000425A0200000000000004E000050032006A
:10CD1000C85A0200000000001A0007000004E000EA
:10CD200003003A00F80007000004E000F4FF3200BE
:10CD300000000600C222A9000001EB0042038800A7
:10CD4000520388000203880012038800F20888005A
:10CD5000ADC0BF00F1C8B30001406000ADE0B70056
:10CD6000E208880000642000D0088800000021004C
:10CD7000506B880080D6200002487800B26A880094
:10CD80000000060080417800006B8000E10F500039
:10CD90007000320003003900E20F5000D8003A0062
:10CDA00076003700E2CF51001000320005003E004F
:10CDB0000304E0000A003200E1CF51005A003A00BB
:10CDC0000F003700F1CF5100CD003200F3CF5100FA
:10CDD000CB003200E4CF510053003A001A00370074
:10CDE000D4FF070010002000C6003700008C280088
:10CDF00050570200000000000000EB00C1003700A7
:10CE0000C222A8000001EB00F2088800B2088800E6
:10CE1000A208880080002000F00888008660A90031
:10CE20009660A900ADC0BF00F1C8B300014060002A
:10CE30000044A000ADE0B70010002000B06A8800F8
:10CE400002007800AF00370010C0B300DC5A0200C7
:10CE500000000000508C2800505702000000000025
:10CE60000040EB00DC5A02000000000010C2B300DA
:10CE7000DC5A0200000000000040EB00DC5A020017
:10CE8000000000000040EB00DC5A0200000000003F
:10CE900000C1B300DC5A0200000000000040EB00BB
:10CEA000DC5A02000000000030C2B300DC5A02006D
:10CEB000000000000040EB00DC5A0200000000000F
:10CEC000F0C0B300DC5A02000000000020C4B30030
:10CED000DC5A02000000000000C4B300DC5A02006B
:10CEE0000000000000C4B300DC5A02000000000093
:10CEF00050C0B300DC5A02000000000010C4B300B0
:10CF0000DC5A02000000000020C0B300DC5A02001E
:10CF1000000000000040EB00DC5A020000000000AE
:10CF20000000EB007700370080D520000348780030
:10CF300041C0B300D0D5200001487800E0D52000E2
:10CF40000048EB0010002000006B88000000EB00A0
:10CF50006C003700E2D520001240E800004978005C
:10CF60000080FB0081D5200003F07800D0D52000A0
:10CF700012417800904F51006100390080D52000A7
:10CF80009040780010C8B30080CF500019003200E4
:10CF900000CCB30080CF50000400320000C8B300C2
:10CFA00080CF500053003A002000370090D5200079
:10CFB000104078008080FB000148A300010032008F
:10CFC0006200A8000138A3000100320062A0A8009E
:10CFD0000128A3000100320062C0A8000118A300CC
:10CFE0000100320062E0A8000008A3000100320046
:10CFF0006300A800A0D520001080FB004800DD00E1
:10D0000091D520009180FB00010070004200DD00FE
:10D0100064004000506B880001002100810F500027
:10D0200034003600516B880032003700B0D5200044
:10D03000104078004800DD0001002000A2D520004B
:10D04000124178000281FB00030020000200700002
:10D0500083807000C808DD000080FD0080407800FB
:10D060000040EB0092D52000124178000281FB00C5
:10D070000300200002007000838070004209DD0080
:10D08000CE00DE00810071004200DD00640040003F
:10D09000E0804800920120000300200024060200E6
:10D0A00000000000106B8800216B8800F00F50001A
:10D0B000E08F58000500360070005000E0805800F6
:10D0C000106B8800216B88000400370010002000DE
:10D0D00001002000106B8800216B8800126B80001B
:10D0E000236B80004018DE0001002000E00888006B
:10D0F000D20888000000EB00006B880001003700B8
:10D100000000EB0000000600B06A8000E10F500054
:10D110002C003A0086C0BF000038A30002003A008D
:10D120006200E20027003A001FE1A8008780A90002
:10D130000000EB00306B8800516B80000100E000C4
:10D140000E00320000017800501680004600DE001C
:10D150007140800000F1780087C0BF000048A30044
:10D16000FDFF32008780A9000201E800516B8000BA
:10D17000810F5100F4FF3900326B88000000EB0092
:10D1800010038800F0088800316B88000100E0007F
:10D1900009003200704080000100400070F89700E4
:10D1A000DC5A020000000000306B80008000E900C3
:10D1B000316B8800F7FF3A00DEFE07001000200008
:10D1C000010037000000EB000000060021D5200020
:10D1D0009180FB008100D10061C160008040780037
:10D1E000024078000901070000102000000006003E
:10D1F00020D520001014A1004101200050EE200095
:10D20000F4730200000000000000060020D520009A
:10D210001014A0002101200090EF2000F473020000
:10D220000000000000000600A0AE20001044A00096
:10D2300020D520001014A000A8C6BF0001CEB30066
:10D24000014060007040B300A8E6B700C9C6BF0047
:10D25000014060007040B300C9E6B700C8C6BF0017
:10D26000014060000034A000C8E6B700CAC2A900AF
:10D27000C8C2A900C902A900C8E2A800C922A90021
:10D28000D0132000101288000000EB00201288004C
:10D290000012880041E2A800D1012000E0F1200046
:10D2A000F47302000000000000000600889FBE002A
:10D2B0008A1F780000047800106480000000E800F5
:10D2C0000080FB0010648800EA19020000000000E2
:10D2D0005418020000000000800478000000EB00F9
:10D2E00020648800E30F54003000320003003E0049
:10D2F0000800E000080032000C003700E60F540080
:10D300003E003200E70F54005C003200E40F54008E
:10D310007A003A00300037008109200000F8200030
:10D32000F473020000000000780037005100200074
:10D3300050602000F4730200000000009500070018
:10D34000E10F5400710032000900E900E10F5000C4
:10D35000110036004102200080012100F473020018
:10D36000000000008001EB002200200011002000DE
:10D3700020002000E41A020000000000E10F50002D
:10D3800003003A000040EB0068000700020037008D
:10D3900080C0B3006500070041002000C0032100E9
:10D3A000F4730200000000005800370011C0B30001
:10D3B0000040EB0095000700F00020002073020001
:10D3C000000000005100200000042100F47302005E
:10D3D000000000004D003700894078000174A00073
:10D3E0000040EB0089000700A1002000500421004C
:10D3F000F4730200000000004400370011C0B300C5
:10D400000040EB0081000700F000200020730200C4
:10D41000000000000900E00004003A0008032000BA
:10D4200009057800090520000900370008032000DD
:10D430000005EB000900E00005003C003300370068
:10D4400090032000800F54000100360008032000E4
:10D450008840780010C0B3006C00070008407800D6
:10D46000DC5A0200000000000804E8000A05E80099
:10D470008A8F5400F2FF3A002400370011C0B30035
:10D480000040EB0061000700F00020002073020064
:10D49000000000000900E00004003A00180220002B
:10D4A000090578000905200009003700180220004E
:10D4B0000005EB000900E00005003C001300370008
:10D4C000F0072000800F54000100360018022000F1
:10D4D0008840780010C0B3004C0007000840780076
:10D4E000DC5A0200000000000804E8000A05E80019
:10D4F0008A8F5400F2FF3A000400370041022000F6
:10D50000E01D2000F4730200000000004F057800C9
:10D510004F04BE0000000600B1002000600B210097
:10D52000F4730200000000000000060002C2B30015
:10D53000824040000040EB0034000700F000200073
:10D54000207302000000000081C0B3000040EB0027
:10D550002E000700F00020002073020000000000F1
:10D5600011C0B3000040EB0028000700F0002000CD
:10D570002073020000000000E1C0B3000040EB0097
:10D5800022000700F00020002073020000000000CD
:10D59000000006000040EB003A000700F000200009
:10D5A000207302000000000031C0B3000040EB0017
:10D5B000220007005000200020730200000000003D
:10D5C00031C0B3000040EB001C000700000A20003F
:10D5D000447302000000000031C0B3000040EB00C3
:10D5E00016000700000A200044730200000000003B
:10D5F00021C0B3000040EB0010000700000A20002B
:10D60000447302000000000000000600889FBE0076
:10D6100080447800014478008180FB00C408DE006B
:10D62000060007006F4464008840780009407800D5
:10D63000020007004F04BE0000000600881F7800AB
:10D64000C408DD00014478000804A000E14F500048
:10D6500002003A00014478003840B30008407800E6
:10D66000080007000834A000084078000500070003
:10D67000084078000034A100020007004F04780041
:10D68000000006004832020000000000CAC2A800E4
:10D69000CAC2A90000000600889FBE008A1F780049
:10D6A000004578008144780040D320000048EB001A
:10D6B0000A04E00003003A00A08120001080A000CE
:10D6C0000C0037000104E0000A003200F1032000E2
:10D6D00050AE2000F4730200000000001101200091
:10D6E000A0192100F473020000000000C85A0200D3
:10D6F000000000004100200040B22000F47302004E
:10D7000000000000CB42A800C942A900310020005F
:10D7100080B220009A73020000000000CBC2BF005C
:10D720004200DE006100600011C0B300F20007009B
:10D73000CB42A900C942A800C222A800C022A90069
:10D7400081002000B0B220009A73020000000000A7
:10D75000C2C2BF000000D1006100600011C0B30070
:10D76000E5000700C222A900C962A800CB62A90097
:10D770008100200030B320009A73020000000000F6
:10D78000CBC2BF004300DE006100600011C0B300E7
:10D79000D9000700CB62A900C962A900810020005E
:10D7A000B0B320009A73020000000000CBC2BF009B
:10D7B0004300DE00610060008040EB00CE00070007
:10D7C000C002A900C202A8002000200020730200AD
:10D7D000000000004100200030B420009A730200D5
:10D7E00000000000C2C2BF006140600011C0B30071
:10D7F000C1000700E100200070B42000F4730200B3
:10D800000000000021E3A8002100200050B5200006
:10D810009A7302000000000072352000712B200076
:10D8200090C0B300710007000904E0000800320056
:10D830003100200070B520009A7302000000000043
:10D8400072352000712B2000B0C0B30067000700C4
:10D8500041002000A0B520009A73020000000000E3
:10D8600002252000011B2000A0C0B3005F000700BC
:10D870000904E0000800320031002000E0B520007B
:10D880009A7302000000000002252000011B200006
:10D89000C0C0B3005500070021E3A90081002000AB
:10D8A00010B62000F473020000000000F8C32F003F
:10D8B0000004FD00C822B6000004FD00003C20006A
:10D8C000CC22B700400620002073020000000000B8
:10D8D00010C0B30061000700A100200090B6200036
:10D8E000F4730200000000000004FD00CC22B6002A
:10D8F0000004FD000904E00002003200C962A80033
:10D90000CB62A90040062000207302000000000046
:10D910000040EB00510007000904E0000B0032005A
:10D92000A100200030B72000F473020000000000C6
:10D93000003C2000C822B7004006200020730200EF
:10D940000000000010C0B300440007000A04E0001B
:10D95000120032000904E00010003200C002A900E9
:10D96000C202A800C422A80001022000D0B72000F3
:10D97000F473020000000000F1002000B018210044
:10D98000F473020000000000C85A0200000000000A
:10D99000C422A900C002A900C202A900D8710200D5
:10D9A0000000000061002000D0B920009A7302003E
:10D9B0000000000048D32000184078002C590200D5
:10D9C000000000008100200030BA2000F473020043
:10D9D00000000000A08120001080A1001880FB0042
:10D9E0004F0578004F04BE0000000600889FBE006F
:10D9F0008A1F7800004478008104780002057800CE
:10DA000080C2B300DC5A0200000000000840780029
:10DA1000167202000000000000047800D8590200CD
:10DA20000000000090C2B300DC5A020000000000B9
:10DA3000890F540003003600100020008A0F5400A4
:10DA4000010039000000EB0011C0B3002A000700FC
:10DA50004F0578004F04BE0000000600881F7800C4
:10DA60000044780041002000B0BA20009A73020000
:10DA700000000000CBC2BF000000D10061006000C8
:10DA8000884078001C00070031002000F0BA200018
:10DA90009A73020000000000CBC2BF00614060002A
:10DAA00088407800140007004100200020BB2000BF
:10DAB0009A73020000000000CAC2BF000080FB0091
:10DAC0004700DE00884078000B000700210020009E
:10DAD00060BB20009A73020000000000CAC2BF00B1
:10DAE0004600DE0061006000884078000200070008
:10DAF0004F04780000000600814F500005003A00F6
:10DB00003100200080BB2000F47302000000000000
:10DB10000600370051002000B0BB2000F473020063
:10DB20000000000040D320001048E800000006007C
:10DB3000408E280050570200000000000000060040
:10DB4000889FBE008A9FBE007940800010002000A0
:10DB5000A06A8800F6FF07008005EB00C85A0200A3
:10DB600000000000E34F50001200320004003E00AD
:10DB7000E14F50003100320034003E009600370083
:10DB8000E64F50000900320003003E00E54F500010
:10DB90008B003A0063003700E74F50003E00320030
:10DBA000E84F500086003A0031003700E0FF0700E0
:10DBB000EAFF370030C0B300804C780080C0B3006B
:10DBC0009044980021E3A800C0C0B3001672020080
:10DBD00000000000C800DE00A1449800B044980096
:10DBE000B0C0B3001672020000000000C800DE00E2
:10DBF000C1449800D0449800A0C0B300167202003F
:10DC000000000000C800DE00E1449800F0449800E5
:10DC100090C0B3001672020000000000C800DE00D1
:10DC2000814C9800904C980021E3A900A1002000AD
:10DC3000090078008E000700C8FF3700C85A0200AC
:10DC40000000000067000700C4FF3700C85A020048
:10DC50000000000000447800C85A020000000000E4
:10DC6000804078000840780091000700BBFF370033
:10DC7000C85A02000000000000447800C85A0200A0
:10DC800000000000C840DD000080FB000080700044
:10DC9000A06A8800B1FF3700C85A020000000000E7
:10DCA0000085FB00E14F500004003A0030C0B30093
:10DCB000F25A0200000000000300370020C2B30047
:10DCC000F25A020000000000C85A020000000000E2
:10DCD00000447800C85A020000000000804078002C
:10DCE000A0CAB300804F540003003A0050C5B300EF
:10DCF00080CF50000400320020C2B300F25A02006C
:10DD0000000000000005EB0070C0B300804C7800FC
:10DD10009A44980021002000090078005400070070
:10DD20008EFF3700C85A020000000000004578004E
:10DD3000C85A020000000000004178008560A90078
:10DD4000C850DD000080FB0000847000000022004D
:10DD5000800F5400010036000004780050C0B3006A
:10DD6000804C78009A449800A2449800310020002A
:10DD7000090078003E0007007040800000408800E5
:10DD8000E7004400C308DE008180400011408800A5
:10DD90002B408800418320008100400031408800F2
:10DDA0004B4088005B4088009560A800A36A800013
:10DDB00008017800B67602000000000067FF370017
:10DDC0008B4C78009B4498001100200009007800DB
:10DDD0002700070061FF37004F05BE004F04BE005B
:10DDE00000000600CAC2A900CB22A900CB02A900EC
:10DDF000CB42A900CA02A900E24F500006003A0037
:10DE0000CAC2A800CB02A800CB22A800CB42A8001F
:10DE1000CA02A80005003700CAC2A900CB02A900A7
:10DE2000CB22A900CB42A900CA02A9000040E90008
:10DE3000E14F500007003E00C8C2A900C922A90056
:10DE4000C902A900C942A900C802A900C8E2A800E5
:10DE500006003700C8C2A800C922A800C902A8004D
:10DE6000C942A800C802A800C8E2A8000000060035
:10DE7000889FBE008A1F7800000578008104780022
:10DE80000100E000070032000004EB0068407D0064
:10DE9000DC5A0200000000000804E800888F5400EB
:10DEA000FAFF3A004F0578004F04BE00000006005C
:10DEB000E44F50002300320005003E00E14F5000C7
:10DEC00008003200E24F50002A003A000D003700EF
:10DED000E84F500021003200F04F500025003A007A
:10DEE00010003700C022A900E1C0600081C04000DE
:10DEF000C2C2BF000014A10001407000C2E2B7001E
:10DF00001C0037000104E00003003200C002A90039
:10DF1000C202A80017003700C002A900C202A9006F
:10DF2000140037000104E00003003200C962A800B9
:10DF3000CB62A9000F003700CB62A900C962A9001B
:10DF40000C003700E1C06000CAC2BF000004A1009D
:10DF500001407000CAE2B70006003700E1C060006F
:10DF6000C208DD00CBC2BF000024A1000140700048
:10DF7000CBE2B70000000600F00F20006C5F02004B
:10DF800000000000000006006C5F020000000000BE
:10DF900080007800A0AE200002C4B30010406100F1
:10DFA00001003A008000EB0001007800000006004C
:10DFB000A0AE20001064A00020AF20001040780028
:10DFC00061406000040032000040EB00D6600200B7
:10DFD000000000000300370010C0B300D66002004C
:10DFE0000000000020AF2000104078006140600079
:10DFF00003003200F0C2B300DC5A0200000000004F
:10E00000A100200090AB2000F4730200000000008B
:10E0100000000600A0AE20001064A10020AF200088
:10E020001040780061406000040032000040EB00C6
:10E03000D6600200000000000300370010C0B300EB
:10E04000D66002000000000020AF200010407800E1
:10E050006140600003003200F0C2B300DC5A0200ED
:10E0600000000000A100200090AB2000F47302002B
:10E070000000000000000600A0AE20001064A10017
:10E0800020AF2000104078006140600004003200A2
:10E0900010C0B300D660020000000000030037008B
:10E0A0000040EB00D66002000000000020AF20001E
:10E0B000104078006140600003003200F0C2B300FD
:10E0C000DC5A020000000000B100200030AC20004B
:10E0D000F473020000000000000006005660020019
:10E0E000000000000080FB0000000600E26002006B
:10E0F000000000000080FB000000060010C0B3001C
:10E1000098600200000000000000060010C0B3008C
:10E11000CA60020000000000000006000040EB00A2
:10E12000CA600200000000000000060010C0B3003A
:10E13000BE60020000000000000006000040EB008E
:10E14000BE60020000000000000006004101200047
:10E15000E0AC20009A7302000000000080AD2000B7
:10E16000104078002C5902000000000000C2B300EB
:10E17000DC5A02000000000020AF200010407800B0
:10E18000614060002C5902000000000000C2B30092
:10E19000DC5A020000000000A0AE20001080FB004E
:10E1A0004400DE00614060002C59020000000000C5
:10E1B00000C2B300DC5A020000000000E08E28001C
:10E1C000685702000000000000000600889FBE00A3
:10E1D000EA190200000000005418020000000000CC
:10E1E00000047800EA190200000000005418020040
:10E1F0000000000080047800EA190200000000001E
:10E200005418020000000000000178000800E90036
:10E21000E30F5000020036000004EB00020037005C
:10E2200080AD20000848E9000900E900E10F500036
:10E23000020036000004EB000500370021AF20008B
:10E240000940E900614060001104A100914870009C
:10E250000200E900E10F500008003E00A0AE2000DF
:10E26000E1406100C408DD00104178000244A100D3
:10E27000014871000800E0002E003A00B1032000C0
:10E2800080452000F4730200000000008001EB00D4
:10E29000420020001100200010002000E41A0200BB
:10E2A0000000000081AD20008048E900D10120007D
:10E2B000601C2100F4730200000000008001EB00EC
:10E2C000220020001100200020002000E41A02009B
:10E2D0000000000021AF20000040E9006140600024
:10E2E0001104A10091487000F1042000E093200087
:10E2F000F4730200000000008001EB002200200007
:10E300001100200010002000E41A020000000000AC
:10E31000A2AE2000614060004400DD009240780021
:10E320000144A10000C970000000EB0020648800D7
:10E330000100370085FF0700A1AE2000F0C9B3003F
:10E340009148600080AD20009040780030C0B3005C
:10E35000AA5E020000000000C922A900C902A900AB
:10E36000C8E2A80020AF20001040780061406000A3
:10E37000D6600200000000004F04BE00000006004E
:10E380000101200040062100F4730200000000009B
:10E3900000000600A1AE20001141780080AD2000F1
:10E3A0000048EB0000CEB30080486100000006008A
:10E3B000889FBE00C922A800C902A800C8E2A80020
:10E3C000C8C2A800C942A800C222A900C022A90050
:10E3D000CAC6BF0009CEB30009406000CAE6B70054
:10E3E0000004EB00A8408800EAFF0700CB62A90008
:10E3F000C962A900C002A900C202A9002D83A90018
:10E400002D43A9002D23A9002D63A9000940780000
:10E410002063B7008819880020F0210020198800A7
:10E42000181988004F04BE00000006000080FB00A1
:10E43000401988002023A8002003A90020C3BF00A2
:10E440000008A300FDFF3200001880000000060055
:10E4500021E3A800C0C0B300F4FF0700D8590200B0
:10E460000000000021E3A90000000600881F7800DA
:10E47000E1002000E0352000F473020000000000FD
:10E48000F1002000B0182100F47302000000000029
:10E49000F1002000C03620009A7302000000000046
:10E4A0000000EB00D859020000000000110020001D
:10E4B000B03720009A730200000000000F00370000
:10E4C00021E3A800C0C0B300D8FF07000004780013
:10E4D00021E3A900A08C2800505702000000000092
:10E4E00008007800D8590200000000001100200048
:10E4F000B03720009A73020000000000425A020068
:10E50000000000000004E000EDFF3200C85A0200E5
:10E5100000000000008D2800685702000000000085
:10E520004F04780000000600881F7800000478007F
:10E5300090AD200010407800EF4F500005003E00E5
:10E540008080FB00EF801000F0FF27000180DE00DC
:10E550000004640090408000E10F5000120032007F
:10E5600005003900E20F50001B003200E30F50009D
:10E5700031003A0026003700A0AE200001C2B300EF
:10E5800010C060000400320008007800AE5902009C
:10E5900000000000280037000800780072590200CF
:10E5A0000000000024003700A0AE200001C2B3002C
:10E5B00010C060000400320008007800E258020039
:10E5C000000000001C003700084078002C590200B1
:10E5D0000000000018003700A0AE200001C2B30008
:10E5E00010C0600006003200084078008857020022
:10E5F0000000000000C2B300DC5A0200000000006E
:10E600000840780088570200000000000A00370028
:10E61000A0AE200001C2B30010C0600003003200B1
:10E620004840DE00DC5A020000000000084078008C
:10E63000DC5A0200000000004F04780000000600D1
:10E64000889FBE008A1F7800000578000000E00067
:10E650000A0034008004EB000004EB00A00F20004F
:10E66000090007000804E800E40F5400FBFF3A002B
:10E670008904E800890F5500F7FF3A004F0578003C
:10E680004F04BE00000006000000E000140034004B
:10E690008000EB000000000000000000000000000F
:10E6A000000000000000000000000000000000006A
:10E6B000000000000000000000000000000000005A
:10E6C000000000000000000000000000000000004A
:10E6D000000000008100E800810F5000EDFF3A00CB
:10E6E00000000600000278008001EB00110020000D
:10E6F000020120008381410001006200010032001C
:10E700000300A000818040000201E900F9FF3A0007
:10E7100090AD200010407800F04F50000300320010
:10E720000080FB00700010008019DE0003007800FC
:10E7300000000600889FBE008A9FBE008100400046
:10E74000810F500025003D000004780039002000B2
:10E750006BFC210001057800110009000904D800B4
:10E760000100E00006003A00000040000B004000FD
:10E770001000BA00DC5A020000000000140037004C
:10E78000E18F500009003A00110009000904D80087
:10E79000000040000B0040001000BA004800DE00FE
:10E7A000DC5A02000000000009003700E28F500030
:10E7B00007003A00110009000904D80000004000D9
:10E7C0000B0040001080BA00DC5A0200000000007C
:10E7D0000804E800880F5500DFFF3A004F05BE002F
:10E7E0004F04BE0000000600D2FF0700208F280063
:10E7F000685702000000000000000600110220001F
:10E8000040272100F8FF0700C10420005029210003
:10E81000F5FF070061022000102E2100F2FF070023
:10E820008102200070302100EFFF0700510120001D
:10E83000F0322100ECFF0700B1012000403421003C
:10E84000E9FF070081022000F0352100E6FF070004
:10E85000B101200070382100E3FF0700E102200031
:10E86000203A2100E0FF070051012000003D210077
:10E87000DDFF070031022000503E2100DAFF0700D3
:10E88000E102200080402100D7FF0700C1012000E5
:10E8900060432100D4FF0700110220002045210021
:10E8A000D1FF0700C101200030472100CEFF070043
:10E8B00051022000F0482100CBFF07001102200088
:10E8C000404B2100C8FF070091012000504D21005E
:10E8D000C5FF0700F1012000E04E2100C2FF070044
:10E8E00091022000D0502100BFFF070051022000FC
:10E8F00060532100BCFF070061032000B0552100D8
:10E90000B9FF0700E103200010592100B6FF0700FE
:10E9100000000600881F7800E100200070912000B0
:10E9200084FF0700C85A020000000000004478007D
:10E93000DC5A020000000000208F28006857020007
:10E940000000000090C7B300804F54000400320064
:10E950008000EB0090C5B300804F540001003A00E6
:10E9600011002000010078004F047800000006002C
:10E9700004000700F4080200000000000000EB00A3
:10E98000000006000400FA00881F7800F0FF2F0046
:10E9900001002000D0BF9F00E1BF9F004507A900F4
:10E9A0002CA3EF004227A9000080EB008080EB0041
:10E9B0005FB99700EFB9970061015100E0815900FC
:10E9C000D2BF9F00E3BF9F005FB99700EFB99700E8
:10E9D000800F5100818F5900F5FF3A00A4C6BF0097
:10E9E00001CEB300014060005040B300A4E6B70080
:10E9F000C4C6BF00014060003040B300C4E6B700A9
:10EA000081C0B30000812000014878000004EB00C1
:10EA100098408800D871020000000000185A0200D7
:10EA20000000000068C0A80068E0A8008800780026
:10EA3000F00F2000025A020000000000B0408800E1
:10EA400021002000F00F2000025A02000000000008
:10EA5000C0408800501680000080FB004200DE00AD
:10EA600063406000E34F500004003A0011C6B30059
:10EA7000A0812000014878000B003700E24F5000D1
:10EA800004003A0021C6B300A081200001487800AC
:10EA9000050037000004E00003003A0051C3B30052
:10EAA000A08120000148780068C0A90068E0A900A2
:10EAB000A08120001080A10081C0B30090AD200093
:10EAC000014878003260EF00A08E280068570200ED
:10EAD00000000000021C0200000000004F0478004B
:10EAE0000080FA0000000600889FBE00C922A8002E
:10EAF000CB22A900C922A90028022000A0002000E2
:10EB000044730200000000000804E900FBFF3A0023
:10EB1000C922A80010042000447302000000000075
:10EB2000CBC2BF00E204600038022000A000200039
:10EB300044730200000000000804E900FBFF3A00F3
:10EB4000CBC2BF00110020000018A300010032005A
:10EB50008980FB00010078004F04BE000000060021
:10EB6000881F780000447800C922A800CB22A900A1
:10EB7000C922A900400020004473020000000000E8
:10EB80000804E00001003200C922A8008000200033
:10EB900044730200000000000804E0000700320097
:10EBA000CBC2BF000000D100614460000002200021
:10EBB00044730200000000000800370090012000AC
:10EBC0004473020000000000C922A8007000200069
:10EBD00044730200000000000044EB0050002000DD
:10EBE00044730200000000000880FB004F0478001E
:10EBF00000000600889FBE000044780089C0B30072
:10EC000061406400D6FF07008880FB000104D1004A
:10EC10000004E000010032000874A0008944E9000B
:10EC2000F7FF3A008000200044730200000000005B
:10EC30000880FB004F04BE0000000600E1C0600039
:10EC400081C04000F52C2000954278000514A100F9
:10EC500081C272008002FD00CFE2B7008002FD0099
:10EC6000616A20009140780005CEB30085C0600045
:10EC70007140B3008000FD00A6E6B7008000FD00F3
:10EC8000916C20009140780085C060005140B30035
:10EC90008000FD00C9E6B7008000FD00C0118800BB
:10ECA0008002EB00851188003062A800614161009C
:10ECB0004411DD0030C2BF000044A10002407000DA
:10ECC00030E2B700E3C1610083C1410030C2BF0040
:10ECD00091CFB300014060000340700030E2B70004
:10ECE0006142620030C2BF000004A1000440700015
:10ECF00030E2B700951188000000060031E2A8005C
:10ED00003342A80087C0A9000000060031E2A90034
:10ED10003342A900F0C1B300A666B700C9C6BF0060
:10ED200001CEB30001406000C9E6B700CF22A900C0
:10ED3000000006008000780033C2BF000018A30066
:10ED4000FDFF3A00A11188000000060032C2BF009A
:10ED50000008A300FDFF3200B01180000000060093
:10ED600032C2BF006100600000000600889FBE0044
:10ED70008A9FBE008C1F78008002EB000203E9002E
:10ED8000800378000104780003067800A92C200095
:10ED90009A0020006B00200010408000E4824200B6
:10EDA0000028E600050078000408E300FEFF3500B7
:10EDB00037017800B70178000280FD000302690086
:10EDC000F40FB20004016900848169000280FD0033
:10EDD000F00020000030E600060078008000780097
:10EDE0000C800900000000001980A1000281D300FE
:10EDF0001950AD008381D3001958AD000C80090073
:10EE0000000000001980A0001970A3000482D30044
:10EE10008100E900F2FF3100EF0010000122DE0066
:10EE2000041C78004300DE000000E8000A28B4005B
:10EE30009580AB0008003200404080000A08E300E3
:10EE4000050032008580A9009580A8000608B4005E
:10EE5000100078002011880070035300CEFF3100AD
:10EE60004F0678004F05BE004F04BE00045B04004F
:10EE70000000000011022000203F2000F473020077
:10EE80000000000010002000206488000000060040
:10EE900011022000203F2000F47302000000000057
:10EEA00010002000206488000010200000000600F0
:10EEB00011022000203F2000F47302000000000037
:10EEC00010002000206488000000EB000000060015
:10EED00011022000203F2000F47302000000000017
:10EEE00010002000206488000000060081C0B300EC
:10EEF00090AD200001487800A0AE20001054A10081
:10EF00000000060081C0B30090AD200001487800E9
:10EF1000A0AE20001054A100000006000101200056
:10EF200040062100F473020000000000000006000B
:10EF3000008F280068570200000000000000060053
:10EF40008080FB000138A30003003200C002A9004A
:10EF5000C202A80002003700C002A900C202A90034
:10EF60000128A30003003200C962A800CB62A900F7
:10EF700002003700CB62A900C962A9000118A300F2
:10EF800003003200C942A900CB42A80002003700AA
:10EF9000C942A900CB42A9000008A3000900320021
:10EFA000A0AE2000104078007040600002003200E7
:10EFB000C8C2A80006003700CCC2A800C8C2A90079
:10EFC00003003700F0FB2F00CC22B600C822B600A9
:10EFD000000006000040DA000000FE00FFFFFF0016
:10EFE000FFFFFF00FFFFFF00FFFFFF00FFFFFF002D
:10EFF000FFFFFF00FFFFFF00FFFFFF00FFFFFF001D
:10F00000FFFFFF00FFFFFF00FFFFFF00FFFFFF000C
:10F01000FFFFFF00FFFFFF00FFFFFF00FFFFFF00FC
:020000040001F9
:00000001FF
